:020000040000FA
:101800000222711A4D1A52227FB8EF90181393904A
:101810001900730A20364CE563FF22EFF563225A64
:101820002D5761766520342E35340002412D000D90
:10183000FA20000DDC7000000000020C00013F3FA8
:101840003F0404041A2A1A347F0322023482C2D5C8
:10185000E830E70FB2D5E4C39BFBE49AFAE499F9C8
:10186000E498F8EC30E717B2D5121884121D02E4A0
:10187000C39BFBE49AFAE499F9E498F88003121DFB
:101880000230D50DE4C39FFFE49EFEE49DFDE49C81
:10189000FC22788CE4F6D8FD9000007F007E10E4F6
:1018A000F0A3DFFCDEFA904FFFA3E583C394204052
:1018B00011FEAF829020000E0FE48002F0A3DFFC47
:1018C000DEFA12192002228322323F241E16110E44
:1018D0000B09070504030201F0C8A791776760466A
:1018E000383532302422201400010102020303049F
:1018F00004050506060707822D1C1613111010FF9C
:10190000C0637419C0E0C082C08375630AE5FF54E8
:10191000CF4490F5FF22C0637419C0E0C082C08339
:10192000756320E5FF54CF4490F5FF22C06374191E
:10193000C0E0C082C083756336E5FF54CF44A0F594
:10194000FF22C0637419C0E0C082C08375634CE598
:10195000FF54CF44B0F5FF229080042116909000F0
:10196000211690900321169097B82116909FAE21D2
:1019700016909FB1211690F9E3211690B7B9211660
:1019800090B7BA211690B894211690ADA021169068
:10199000C004211690C01C211690C022211690A6CA
:1019A00015211690C3142116909922211690C50F67
:1019B000211690C524211690C536211690C5CB213D
:1019C0001690C553211690C741211690C7AF211616
:1019D00090C817211690A217211690A0B921169031
:1019E000A0D2211690A014211690C8AE211690A85E
:1019F00059211690A7A5211690AFAA211690C8F0DC
:101A0000211690A299211690A1C9211690A10A2110
:101A10001690A180211690CA32211690CB4821162B
:101A20009097D7211690CA78211690CC372116901E
:101A3000BD80211690CDAE211690C9CA211690C73F
:101A40003B211690C677211690C683211690CEBDF5
:101A50002116909E31211690C79B211690A77821C0
:101A60002C90824A212C908000212C90A7FF212CC1
:101A700090A82B212C9081C5212C90A84B212C9033
:101A8000AC82212C90AD5E212C90ADD6212C90AE55
:101A900002212C90993A212C90834A212C90AE1946
:101AA000212C90830F212C90AE5F212C00BB0106CE
:101AB00089828A83E0225002E722BBFE02E3228968
:101AC000828A83E49322BB010CE58229F582E583B7
:101AD0003AF583E0225006E92582F8E622BBFE06AD
:101AE000E92582F8E222E58229F582E5833AF58349
:101AF000E49322BB010989828A83F8E028F022500E
:101B00000327F722BBFE05F8E328F3228A838982A4
:101B1000F8E4932822BB010689828A83F0225002CE
:101B2000F722BBFE01F322F8BB010DE58229F58205
:101B3000E5833AF583E8F0225006E92582C8F622CB
:101B4000BBFE05E92582C8F222EF8DF0A4A8F0CFF4
:101B50008CF0A428CE8DF0A42EFE22BC000BBE007B
:101B600029EF8DF084FFADF022E4CCF875F008EF9A
:101B70002FFFEE33FEEC33CFEE9DEC984005FCEEEC
:101B80009DFE0FD5F0E9E4CEFD22EDF8F5F0EE84F0
:101B900020D21CFEADF075F008EF2FFFED33FD40B5
:101BA00007985006D5F0F222C398FD0FD5F0EA222F
:101BB000C2D5EC30E709B2D5E4C39DFDE49CFCEE50
:101BC00030E715B2D5E4C39FFFE49EFE121B5BC352
:101BD000E49DFDE49CFC8003121B5B30D507C3E44D
:101BE0009FFFE49EFE22C5F0F8A3E028F0C5F0F8C0
:101BF000E582158270021583E038F022A3F8E0C573
:101C0000F025F0F0E582158270021583E0C838F007
:101C1000E822BB010A89828A83E0F5F0A3E0225022
:101C20000687F009E71922BBFE07E3F5F009E3197F
:101C30002289828A83E493F5F074019322BB010A1E
:101C400089828A83F0E5F0A3F0225006F709A7F015
:101C50001922BBFE06F3E5F009F31922EF2BFFEE84
:101C60003AFEED39FDEC38FC22C3EF9BFFEE9AFE05
:101C7000ED99FDEC98FC228E8FF0A4CC8BF0A42C77
:101C8000FCE98EF0A42CFC8AF0EDA42CFCEA8EF08A
:101C9000A4CDA8F08BF0A42DCC3825F0FDE98FF071
:101CA000A42CCD35F0FCEB8EF0A4FEA9F0EB8FF068
:101CB000A4CFC5F02ECD39FEE43CFCEAA42DCE35F0
:101CC000F0FDE43CFC2275F008758200EF2FFFEE7A
:101CD00033FECD33CDCC33CCC58233C5829BED9A58
:101CE000EC99E58298400CF582EE9BFEED9AFDECB6
:101CF00099FC0FD5F0D6E4CEFBE4CDFAE4CCF9A8FC
:101D00008222B800C1B90059BA002DEC8BF084CF03
:101D1000CECDFCE5F0CBF97818EF2FFFEE33FEEDDA
:101D200033FDEC33FCEB33FB10D703994004EB9904
:101D3000FB0FD8E5E4F9FA227818EF2FFFEE33FE17
:101D4000ED33FDEC33FCC933C910D7059BE99A404C
:101D500007EC9BFCE99AF90FD8E0E4C9FAE4CCFB64
:101D60002275F010EF2FFFEE33FEED33FDCC33CCB8
:101D7000C833C810D7079BCE9AE899400AED9BFD5F
:101D8000EC9AFCE899F80FD5F0DAE4CDFBE4CCFA54
:101D9000E4C8F922EF5BFFEE5AFEED59FDEC58FC6A
:101DA00022C3E49FFFE49EFEE49DFDE49CFC22EB45
:101DB0009FF5F0EA9E42F0E99D42F0E89C45F02252
:101DC000E8600FECC313FCED13FDEE13FEEF13FF01
:101DD000D8F122E8600FEFC333FFEE33FEED33FDA1
:101DE000EC33FCD8F122BB010789828A83021E28CA
:101DF0005005E9F802204BBBFE05E9F80220572206
:101E0000E0FCA3E0FDA3E0FEA3E0FF22E493FC746A
:101E10000193FD740293FE740393FF22E0F8A3E0A4
:101E2000F9A3E0FAA3E0FB22ECF0A3EDF0A3EEF0BF
:101E3000A3EFF022A8828583F0D083D082121E4BBC
:101E4000121E4B121E4B121E4BE473E493A3C58368
:101E5000C5F0C583C8C582C8F0A3C583C5F0C583D6
:101E6000C8C582C822A42582F582E5F03583F583B2
:101E700022E0FBA3E0FAA30EF922F8E0FBA3A3E023
:101E8000F925F0F0E582158270021583E0FA38F04A
:101E900022EBF0A3EAF0A3E9F022BB010789828AD2
:101EA00083021E715005E9F8022063BBFE05E9F8C4
:101EB00002207589828A83022087BB011A89828A5F
:101EC00083D0F0D0E0F8D0E0F9D0E0FAD0E0FBE841
:101ED000C0E0C0F0021E915016E9F8D083D082D045
:101EE000E0F9D0E0FAD0E0FBC082C08302206CBBF6
:101EF000FE16E9F8D083D082D0E0F9D0E0FAD0E045
:101F0000FBC082C08302207E22D083D082F8E4937B
:101F10007012740193700DA3A393F8740193F5826A
:101F20008883E4737402936860EFA3A3A380DF8ABD
:101F3000838982E473EC8EF0A4CCC5F0CCCDF8EFAD
:101F4000A4CEC5F02DFDE43CFCE8A42EC8C5F03DB0
:101F5000FDE43CFCEFA4FFE5F028FEE43DFDE43C9D
:101F6000FC22E709F60870FA8046E709F20870FAE1
:101F7000803E88828C83E790F0A370FA807EE3092C
:101F8000F60870FA8076E309F20870FA806E8882AB
:101F90008C83E309F0A370FA806289828A83E0A3CC
:101FA000F60870FA805689828A83E0A3F20870FAF4
:101FB000804A80D280FA80C680D4806580F28031E9
:101FC000801080A680EA809A80A880DA80E280CAA9
:101FD000803189828A83ECFAE493A3C8C582C8CC95
:101FE000C583CCF0A3C8C582C8CCC583CC70E980BA
:101FF0000D89828A83E493A3F60870F9ECFAA9F0BC
:10200000EDFB2289828A83ECFAE0A3C8C582C8CCA2
:10201000C583CCF0A3C8C582C8CCC583CC70EA8088
:10202000DD89828A83E493A3F20870F980CE88F078
:10203000ED2402B4040050C4F582EB2402B4040081
:1020400050BA2323458223901FB273ECF608EDF6B5
:1020500008EEF608EFF622ECF208EDF208EEF208D0
:10206000EFF222E6FB08E6FA08E6F922EBF608EAC8
:10207000F608E9F622E2FB80E2FA08E2F922EBF246
:1020800008EAF208E9F222E493FB740193FA74027D
:1020900093F92241257D004102B2004127B900C1D8
:1020A00027C11F4104150601140041041401410415
:1020B0001301C118011A00011700C119C11BC10F7A
:1020C000412379004123DFFF4123D700C10EC10D19
:1020D0004123E0004123E1004123D801C111412304
:1020E0007800C11EC115013000C112C1134326E1A1
:1020F0000000004126E0004126E40049229E4C6990
:1021000066656C696E65004622A7424153494300EB
:10211000C1074122B500C108C1094122B6004222CF
:10212000B700004122BB00C10AC10B4122BD0141E1
:1021300022BEFF4122C2024122C3034122C7004105
:1021400022C8004122CA004122CB004122CE0041D8
:1021500022CF004122D0004122D1004122D20041B1
:1021600022D3004122D6004122D7004122D800418B
:1021700022D9004122DC001422DE004122E000418D
:1021800022E1004122E2004122E3004122E4004139
:1021900022E7004122E8004122E9004122EA004111
:1021A00022EB004122EDFF4222F100004222F30027
:1021B000004122F7004122F8004122FD004122FFA8
:1021C000004123000041230100412302FF41230479
:1021D0000541230D0A41231FFF412320C441232130
:1021E00040412325FF41236F00E00C026030001EB8
:1021F000010A00040001010A043600902093E47EE5
:102200000193700122A3FF543F30E509541FFEE4FF
:1022100093A360010ECF54E0B4E03AEFFAEEF9E494
:1022200093FBA3E493FEA3E493FFA3E493FDC08395
:10223000C082C001C002C006C007121971D007D009
:1022400006D002D001D082D083A30FEF70010EDA46
:10225000DAD9D880A954C025E060105005A3DFFD6D
:10226000809CA3A3A3DFFDDEFB8093A3A3DFFD80FF
:102270008D75818C75FF03579E02121920022A4921
:102280000218C8902093E47E019360F4A3FF543FAA
:1022900030E509541FFEE493A360010ECF54E0B46F
:1022A000E00EEFFAEEF9A3A3A3A3DAFDD9FB80D6E3
:1022B00054C025E0604B5026E493A3F85407240C47
:1022C000C8C333C4540F4420C8834004F45680016B
:1022D00046F6DFE480B00102040810204080E49359
:1022E000A3FAE493A3F8E493A3C8C582C8CAC5833C
:1022F000CAF0A3C8C582C8CAC583CADFE9DEE780C1
:1023000085E493A3F8E493A34003F68001F208DF89
:10231000F40222865E7131337286598570775A7A5B
:1023200073EF201A6B1A701A751A7A1A7F1A841AA8
:10233000891A8E19D519DA19DF19E419E919EE1974
:10234000F81A07A104197B198A198F199419991978
:10235000A37F01B1C9902575E0121F0923780423DA
:102360008014238515238A17239A30239F3423A4AE
:102370003623A937000023295357EF855780802F34
:102380005358EF80085358DF800353587F85589087
:10239000801D5359DF8559A08015535AFE800D5377
:1023A0005AEF8008535ABF8003535A7F855AB07F33
:1023B0000CDFFE227F01B1C99027B67401F090278F
:1023C000B6E0602E912E914B9027B6EFF091EC91F4
:1023D0003A902571EFF091EC9027B6E05401F1416D
:1023E00060DCA3E0F460D7EF30E7D3E49027B6F0E9
:1023F00080CC71557F9F9132914B9025729149907D
:1024000025779149902578EFF0B1C5902570E0F4DB
:10241000601BA3E0F46016902577E0FD541F240FA5
:10242000A3F0EDC41354074480902577F022715532
:102430007F05E5C820E2FB8FEB2271557FD79132F3
:102440007FFF9132914F902570EFF07FFF9132E541
:10245000C820E2FBAFEB227F01B1C9302514912ED9
:10246000914B9027B8EFF091EC9027B8E020E00274
:10247000C225302517913A092571EFF141600BA370
:10248000E0F46006EF30E702C22591ECE4FFB1C949
:10249000A225E433FF229026F7121E289026F71279
:1024A0001E00B1D59026FBE06F6033D1B69157EF97
:1024B0006004D1A280F791E07155D1C560079026E4
:1024C000F7F10D91329026F7F10391329026F71231
:1024D0001E00E491329026FBE0FFB1C3D322C32259
:1024E0007F01B1C9D22571557F069132F1DEEF70BF
:1024F000FB902577E0F4600A9027B57406F0F11799
:1025000070FC902575E0121F09252504252D142542
:102510003215253717254730254C34255136255699
:10252000370000253F435710855780802F435810B0
:1025300080084358208003435880855890801D436D
:1025400059208559A08015435A01800D435A1080A7
:1025500008435A408003435A80855AB09027B57487
:102560000CF0F11770FC22902632121E28902636AD
:10257000121E91D1B69157FE6004D1A280F791E06E
:102580007155D1C56007902632F10D9132902632F7
:10259000F1039132902632121E00E4801C902639FD
:1025A000F1526019902636121E71EA494B6008906C
:1025B0002636E4F1498001E4FF913280E091ECE4B9
:1025C000FF8006913291ECE4FFEFB4010443FE205A
:1025D0002253FEDF229026F2121E28D1B69157EF29
:1025E0006004D1A280F771517F03D1CA60079026A1
:1025F000F2F10D91329026F2F10391329026F2120F
:102600001E00E49132914B9026F6EFF0B1C5902672
:10261000F6E0FF2290263B121E2890263F121E91C4
:10262000D1B69157EF6004D1A280F771517F03D1E9
:10263000CA600790263BF10D913290263BF1039141
:102640003290263B121E00E49132902642F15260F5
:1026500014914B90263F121E71EF121B15902640CD
:10266000E4F1E480E591ECE4FFA1C9D1B69157EF24
:102670006004D1A280F7910E71557F0191327F03E2
:10268000913291ECE4FFA1C9902570E020E0127135
:10269000517F3D91327F2A91327F8091327FA6B166
:1026A000C322E51530E20EE51520E509E51530E019
:1026B000047F01F17E2275FF02E5E430E10675E456
:1026C0000675E40322902573E0FF9132902576E0B1
:1026D0006402229027B7EFF090257EE0640270221A
:1026E00071519027B7E07FAB60027FB9913291ECD6
:1026F0009027B7E090257DF070047F1EDFFEE4FF99
:10270000B1C922121E007808121DC0E422121E0058
:102710007810121DC0E4229027B5E014F0E022D119
:10272000B69157EF6004D1A280F722E075F002A4C1
:102730002481F9740F35F07B02FEAF01E4FCFDA1AA
:10274000D5F0902570E0FFF42275F001121E7A0298
:102750001AAD74FFF5F0121BFC45F0229026BEF175
:10276000EAC0079026BE121E719026C1E0FF902697
:1027700042E4F0A3EFF0D070C114EFF07F01EF60FE
:102780000C122CB9AE83E4FD1234048009F1BA12A4
:1027900047C8E433FF227F012290043F121E91C2FA
:1027A00028E4FFF17EBF010B90043F121E71123C22
:1027B0009992287F01F17EA22822F1C5EF700512BF
:1027C0002CC980F622E4FFF1F154F0FEBE40037FF5
:1027D00000220FEFB403F07F0122E4FFA1C9E5C896
:1027E0005404FF2275F001021BE6121E91E4FCFD69
:1027F0002275F0E5EF900001121E65E0229025722F
:10280000E0121B15902577E0900001121B27902500
:1028100078E0900002021B277A2579757F03D1FCAE
:102820007A25797E7D017F081219C67A25797B7F0A
:102830000931DB7A2579797F0B31DB902579E0FE50
:10284000A3E0FF4E6006BEFF1BBFFF1890257EE091
:1028500024FD600304700431E28009902579E4F0DE
:10286000A37440F090257EE024FD6003047008907E
:1028700025767403F080060925767402F09025759C
:10288000E0121F0928A00428AB1428B31528BB1791
:1028900028D13028D93428E13628E937000028C665
:1028A00075FF015353EF8553FD804775FF01535466
:1028B000EF800E75FF015354DF800675FF015354FE
:1028C0007F8554C9802C75FF015355DF8555CA801B
:1028D0002175FF015356FE801675FF015356EF8098
:1028E0000E75FF015356BF800675FF0153567F8555
:1028F00056CB1224EC7F1131CDE4FF1226D31223E4
:10290000B49025737402F0902577E0247F60090469
:10291000701631D3740A800712268831D37458F0A8
:102920009025767403F031E2902578E0F46002217E
:10293000CA90257BE0FEA3E0FF64104E7006902550
:1029400078740EF0EF64204E7006902578740FF0C6
:10295000EF64404E70069025787410F0EF64804E5E
:1029600070069025787411F0E4B5070AEEB40106FC
:102970009025787412F0E45B070AEEB40206902505
:10298000787413F0E4B5070AEEB404069025787461
:1029900014F0E4B5070AEEB408069025787415F033
:1029A000E4B5070AEEB410069025787416F0E4B585
:1029B000070AEEB420069025787417F0E4B5070AEC
:1029C000EEB440069025787418F002266BEF442090
:1029D000F5FE227F1031CD902573227B017D02020E
:1029E00019C69025797401F0A3E4F0221118124C55
:1029F0002E1219AD1242439002B3E064017F0060D1
:102A0000027F01121A16121A1B1219851255CF795C
:102A1000B6121962D1F5E0FE4FFDA3E0FC4DFDA317
:102A2000E0FB4D600BEE5FFFEC5FFFEB5FF47002CD
:102A3000D1A690121CE0FF540324B6F582E43402C0
:102A4000F583E06F9002B1F02275FF0275E404E4B3
:102A5000F5E4C21775FF02901215E0603CE5E654FC
:102A60000364017034121A3E1249D240209012229F
:102A7000E0600DE014F07080121892E4901215F0EE
:102A8000901215E07002611012399C6110121892B8
:102A9000D217E4901215F08077121892124CFA9027
:102AA00002B3EFF0901200E0B47A14901214E0B484
:102AB0009C0D9002B3E0FF64056004EFB4032EE4C4
:102AC0009002BCF09002BCE0FFC394405013E42F8E
:102AD000F582E43412F583E4F09002BCE004F08067
:102AE000E3901200747AF0901214749CF01219CBD7
:102AF0007B017A1279107D017F011219C67A127951
:102B0000117F21D1FC7A1279127D017F221219C620
:102B1000121A43124CFA1240CA9002B3EFF0121983
:102B2000B71240859002B3E0FFB40602800C301764
:102B3000047F0280059002B3E0FF121A5CEF24FFCD
:102B4000B3922775FF0253E6BF9002B3E0640160C1
:102B500005E4901215F0124111121A4831EC90124E
:102B600015E0700F20270C121A667B017A2379E397
:102B70001219FD90121DE003E00280033017057F5B
:102B80000112277ED2AF302775F1B812439B121A7B
:102B9000611219C140F39002B2E0603EF11FEF7084
:102BA00004F1434035E51470FCE51520E5031247B8
:102BB000C812195DEF70FAF1315004F18B50057FA6
:102BC000011226D39002B2E0B40204E4FF8009901F
:102BD00002B2E0B403047F01F1D491C9E51530E1FC
:102BE000A8D1774002E4F0E51520E50991B9AE835C
:102BF0007D011234049002BC91BCF106808B12401E
:102C000015F19F5002D1A69002B2E0605A9023794C
:102C1000E07054F11FEF7004F143404BE51470FC79
:102C2000E51520E50A90121DE020E0031247C812C6
:102C3000195DEF70FAF1315004F18B50057F0112EC
:102C400026D39002B2E0B40203E480189002B2E00E
:102C5000B403047F01800E9002B2E0B40509901223
:102C6000157401F0FFF1D4F1B812439B121A93903E
:102C700002B0E0700491C90815124051FF9002B0F3
:102C8000E0FEC3EF9EC394064002E4F0D2AD1218FA
:102C900007E51530E11BD1774002E4F0E51520E5AA
:102CA0000991B9AE837D011234049002BC91BCF14C
:102CB00006121A2F12407061FE9002B4E075F0AA5D
:102CC0009002BF121E65AF8222E4900449124CBBF1
:102CD00075F0E5E5621227F554F064407002C122F8
:102CE000E4FE75F0E5EE1227F5FDB4010990044A03
:102CF000EEF0E4FF8023EDB4020B90044AE0B4FF51
:102D000004EEF0800F75F0E5EE1227F554F0FDBDEE
:102D100080027F010EEEB403C9EF600690044A748E
:102D2000FFF090044AE0F47002C1221244B1500254
:102D3000C122E51530E102C12290044AE0FF900073
:102D400004D18C30E408900006D194549FF0D165F2
:102D50009000B8121E65E0540FFEBE05089000BC3E
:102D6000D19430E114D165900003121E65E020E596
:102D7000289000BBD19DB4FF2090044AE075F0E597
:102D8000900005121E65C083C082E04401FFA3E0ED
:102D9000D082D083CFF0A3EFF090044AE0FD900002
:102DA00005D18CFEA3E0FFC006C007ED75F0E5A4D9
:102DB00024B3F9740035F0FA7B01C002C001D1657B
:102DC0009000D9121E65E090042CF0EF75F0E5A498
:102DD0002409F9740035F0FAA3121E91D165900010
:102DE000B2121E65E0900430F09000DAD19D90049C
:102DF00031F0E4A3F0D001D002D007D00612318C1C
:102E0000502090044AE0F56275F0E51227F5444041
:102E1000F09004497401F090200EF0E51530E202C4
:102E2000D322E51530E2377F04D16E75F0E5E56217
:102E30001227F5FF54F06440701F75F0E5E562124B
:102E40004CB3540FF075F0E5E5621227F54480F0BD
:102E5000E562F11012198080057F0112277E90042F
:102E600049E024FF2290044AE0FF75F0E522C2AF5A
:102E7000EFF45215D2AF22F702D16E9002B4E09077
:102E800002BCF09002B404F0C394022275F0E51283
:102E90001E65E02275F0E5EF121E65E02275F0E593
:102EA000EF121E65E022E4FF12277EEF60467B01F1
:102EB0007A0279B61227999002B6E0C394C040EE28
:102EC0007B017A0279B8122799D1F5E05FFFA3E080
:102ED0005FFFA3E05FF460E890121DE030E0057F43
:102EE0000112277EE490121CF07B017A0279B6E091
:102EF000FD121967229002B6E0FFA3227B017D013B
:102F00001219C67B0122AE839002B5E0FD0219A81A
:102F100075F0E5A42401F9740035F0FA7B0122E490
:102F2000FF1227F160037F00220FEFB403F37F014C
:102F300022900001740193B40007E493B41802C313
:102F400022D3229002BDE0FEA3E0FFF155D3EF941F
:102F5000C8EE940022902795EEF0A3EFF01244966D
:102F60009027951255DE5009C3EF9DFFEE9CFE8021
:102F700019902795E0FCA30EF4FDECF4FCED240180
:102F8000FDE43CFCED2FFFEC3EFE227F017E009035
:102F900017FCE4935EFE7401935F4E24FFB322900E
:102FA000121CE07011D1F5E04FFFA3E04FFFA3E04A
:102FB0004F7003D38001C322302018E560601415E0
:102FC00060902793E0FEA3E0FF4E6007AA06A907E2
:102FD000121F2F2243FB1075FF0243E640EF600DE6
:102FE00075FF02E5E120E7FB43FB0D800343FB0E89
:102FF00080FEFEAF01E0FDAB05E4FCFD9026FBEB9F
:10300000F0022496123114121E919025ED121E71B9
:103010009025F012389B9025E9121E0012380150BD
:103020000201CA90257AE024FFFF902579E034FF61
:10303000FEE4FCFD9025E9121E1C121D949025F261
:10304000EEF0A3EFF04E603311CCC390257AE09FF1
:10305000FF902579E09EFE9025F2F0A3EFF09025F9
:10306000F01255DE5002313611D5121E71E94A6058
:103070000411CC80487E00F70080429025F0E0FEED
:10308000A3E0FF4E6042902579E0FCA3E0FDD3EF82
:103090009DEE9C400A9025F2ECF0A3EDF0800D909F
:1030A00025F0E0FFA3E0A3CFF0A3EFF011D5121EAF
:1030B00071E94A600411CC80047E007F009025EE07
:1030C000EE8FF0121BE680B3D322C3229025F2E0EC
:1030D000FEA3E0FF229025ED121E719025F2E0FF85
:1030E000A3E0902639CFF0A3EFF09025E9121E005F
:1030F0001225679025F2E0FEA3E0FFC39025F1E0E2
:103100009FF09025F0E09EF09025E9121E1CE4FC53
:10311000FD121C5C9025E9121E289025ED229026B8
:10312000781227EAC007902678121E7190267B122B
:103130005411D0070104A3ECF0A3EDF02290043C5D
:10314000EFF03136751401E4FBFDFF714E7B017A1F
:1031500004791671B1E4FD7F02F1B9125600F5D27F
:103160009004167455F090043CE0900417F090041D
:10317000147402F090043E0E90042530E507E4F04C
:10318000A3743CF022E4F0A374F0F0229004271220
:1031900055C6C2EBE51460026132E51530E202C3A8
:1031A00022F1F15004C22F71BED11EE5D120E0FB07
:1031B000E4F510C217900428E05407C39403E49484
:1031C000005022900430E0FF90042CE02FFFE43305
:1031D000FED3EF9440EE648094804009431504A22E
:1031E0001692EDD32290042D121E71CFE9CF8A11D1
:1031F0008F12900430E0F516AE11124DEB900429B9
:10320000121E718B1C8A1D891E90042CE0F51F90E4
:103210000427E0FCA3E0FD54606031900431E0FF3E
:10322000313D7140121AADFB7A00900425E0FEA3F7
:10323000E0FF7C007D17121B49EF2BFFEA3EFEEFFB
:103240002414FBE43EFA7D027F016114900427A35D
:10325000E05407900414F0751408900429121E71AC
:1032600071B190042CE0FFAD16F1B9900414E06444
:103270000370277B01FD71D3718250077140740187
:10328000121AF3E4F5FF1256137140121AAD2428F6
:10329000FBE433FA7D03E4FF807A900414E06402D7
:1032A0007023713A71824007714074FF121AF31251
:1032B0005600F5D27140121AAD2414FBE433FA7DA6
:1032C000027F01804FE4713A71824007714074FFC0
:1032D000121AF3E4F5FF71A67F0560027F0AEF542E
:1032E0007FFFE5D254804FF5D2E4F5FF43D28071E1
:1032F00040121AADFD7C0071A67E0060047F0A803A
:10330000027F05EF25E0FFEE33FEEF2DFBEE3CFAEA
:103310007D017F01124B73900427E0FEA3E0FF12B2
:1033200045644006A21692EDC322A21692EDD2EB9E
:10333000D322A21692EDD2EBC322FB7D01FF714E88
:10334000900429121E71E92407F9E43AFA22E4F5FF
:10335000FF75D102E5D120E0FBE4F5FFF5D1EF6088
:1033600008E4F5FF43D2808006E4F5FF53D27FEBFB
:103370006006E4F5FF43D140ED6006E4F5FF43D17C
:103380000822121AADFF900430E0FD90042CE02DCD
:10339000FDE433FCED2401FDE43CFCD3EF9DEC6443
:1033A00080F874809822900427E0FEA3E044104E39
:1033B00022E4F5FFE9124DE2EA540F42D6229027AB
:1033C000BAE5F4F0E0547FF5F47F827E00F116F167
:1033D000A25005E5FC20E6F7302F089027BAE0441C
:1033E00080F5F47FE87E03F116F1A25005E5FC209C
:1033F000E6F775FF01E5D520E702C322E5F4D330F7
:10340000E601C322900439EEF0A3EFF0E5147071E9
:1034100012561CF1F15004C22F71BE900439E0FE27
:10342000A3E08E11F512AE11AF127DAA124DC1E4C8
:10343000F5FF75D901F510E5155421602BE5153020
:10344000E504E4FFD12AE490043BF090043BE0045F
:10345000F0124A2EEF600990043BE0C3941040EB59
:103460007F02121AA75315DE900413E07F00B40305
:10347000027F01D12AB1E92D2F71BED2EBA21692A3
:10348000ED22C0E0C0F0C083C082C0D075D008C0BB
:10349000FFF1478F18E51864027050E51424F860B6
:1034A0004024076002A1DC90042512441B7028AB65
:1034B0001CAA1DA91E71B1AD16AF1FF1B9E4FB7DA9
:1034C00001FF714E75FF0012561343FA0475FF0099
:1034D000B1EF751408A1DC43FA0475FF00B1EFA148
:1034E000DCC2EB751400431504A1DCE5186401602F
:1034F00002A1DC12507B4002A1DCE510702B85128A
:1035000082851183E090044BF0E0FF64556004EF86
:10351000B4540BD217124053900424F0A1AB751091
:103520000275FF0075D908A1DCE5106402705A121B
:1035300055F6F583E090044BF012500E1247FD90C3
:103540000413EFF090044BE0FFD39409402590045E
:1035500013E0D39402400CEFD394AA7F0040027F83
:1035600001800D90044BE0D394407F0040027F0126
:10357000EF6005124822803390044BE0FFF516758A
:10358000FF008FD97510038053E5106403704D124E
:10359000482275FF00900413E0C39403E5D350055F
:1035A0005402FF80035401FFEF6004B1F6802DC286
:1035B0002F71BE75FF00D121E5D120E0FBC2EB43A6
:1035C0001502751000900413E0B4030A1516125585
:1035D000F6F583E516F09002B5E516F0D0FFD0D0F1
:1035E000D082D083D0F0D0E03243FA04E4F5FF5328
:1035F000D1FD43D10122D11AE5D120E0FBE4F5FF52
:1036000075D901900413E07F00B403027F01D12A31
:10361000B1E9D22F71BEE4F51022C22F71BEE4F5DC
:10362000FFE5D154FE4402F5D12275FF01E5D53006
:10363000E602C322E4F5FF439A80EF123FE3E4F58C
:10364000FF539A7FD322902743EFF0A3123F38E92C
:10365000F075FF01F147EF64016002C322E5F43029
:10366000E602C3227FE87E03F11AF10FF1DB40018D
:1036700022C22F71BE902734E0FFD12A53F4DFD24B
:103680002F71BE7F787E00D1C975FF0153E4BFE57D
:10369000E430E7FB124B087F8A12560A30E6061226
:1036A0003ED9E4800875FF01123ED9E5D9121B15F9
:1036B00075FF0143E44090120EE0D39401400343B0
:1036C000F420F1DB400122D322CDEFCDCCEECCF1C2
:1036D000ADAB94EF4BF1F9CBEFCBFAE59130E71DB1
:1036E000F1B0A994E9F582EF4582FFEB2DF582EA6E
:1036F0003CF583C3EF9582E5F0958340DEE59120AC
:10370000E708CEECCECFEDCFF13A227E00F11A756C
:10371000FF0343918022F17180F575FF03D3EF948D
:1037200002EE9400400874FE2FFF74FF3EFEEFF59A
:1037300092EE540FF591227F3FFEF11AF10F75FFC3
:1037400003E59120E7FB227FFAF10BE5FC30E6046C
:10375000F1A240F7E5FC30E6037F032275FF01E5A7
:10376000D530E6037F0222E5D57F0030E7027F01F6
:1037700022902733EEF0A3FEF07B017A277935F112
:10378000C65014902735E0FEA3E0FF902734E09F59
:10379000902733E09E400A902733E0FEA3E0FFF13C
:1037A0001A2275FF03E591C330E701D32275FF03A9
:1037B000AF93EF75F010A4FF22E4F5FF8FD4F5FF6F
:1037C000CFEDCF8FD522F1ADAD94EF4DF1F98FF064
:1037D000121C3DE591C330E701D322E5F730E50F38
:1037E000E5F754C07004F1A240F1123F31C322D377
:1037F00022E5F4C330E701D32224FBFFE5F034FFD8
:10380000229024D4121E289024D8121E91E49024D1
:10381000FBF0D39024DCE0941E9024DBE094004085
:1038200001227B017A2479DD9024DBE0FFA3E09084
:103830002642CFF0A3EFF09024D4121E00122614DB
:103840009024D8121E71E94A600F9024FBE0F582A3
:10385000758300121AC6FF80027F009024FBE024CB
:10386000DDF582E43424F583E06F6002C322902406
:10387000FBE004FFF0D39042DCE09F9024DBE09477
:103880000050BD2290267F1227EAC00790267F12A3
:103890001E71902682119BD0070101E0FFA3E090EA
:1038A00024DBCFF0A3EFF022E4F97D0CAC0109ECAE
:1038B00090181F93FC0FEFAA0670010E14F5828A70
:1038C00083ECF0DDE70218488F828E83E4F0A37466
:1038D0000411DB743611DBA3E4F022F08F828E83B7
:1038E000A3A32275FF0275E40475E40175E40222C6
:1038F00075FF0275E404E4F5E42290043331C790C7
:10390000121DE05430600631C45002C322900433CB
:10391000E0B4040BA331619004337403F08025906C
:103920000433E06405701890121DE090043430E513
:103930000631617F1F80043169E4FF31BC8005904E
:1039400004343169900433E09002B2F0900435E021
:10395000901222F01244969002BDEEF0A3EFF0D345
:1039600022E0FB7D017F018006E0FB7D01E4FFEBAF
:10397000600875FF0153CDDF800675FF0143CD025E
:10398000ED600553FBDF800343FB20EF600775FF0D
:103990000243E1402275FF0253E1BF2290121DE075
:1039A0007B027D0130E5087F01316F7F1F8006E4D7
:1039B000FF316FE4FF31BC7F01022FD475FF028F0E
:1039C000E32280F8A21722EFF0A3EDF0A3EBF022A0
:1039D00090269231C79026987401F0C22E7FE87E1F
:1039E000031237161237A25005E5FC20E6F612370F
:1039F00047BF0108E4F5FC75FC408008123747BF5B
:103A00000202D322F1D5902693E0FF124FD975FF21
:103A10000153D5DF53FAFB902692E0FF12362A902D
:103A20002693E0902692B40809E051E12452918E49
:103A30008004E051E1FFD18C902694E0FFF1C8753D
:103A4000FF0175FF03759B047FE87E03123716752F
:103A5000FC42E5FC20E1051237A240F3902695E0F8
:103A6000F075FF03E59B20E7051237A240F3E59BC5
:103A700020E70C75FF0375B91FF115D22E804DD1CB
:103A800085D1E5902693E0FD90120FE05D701C90CB
:103A90002692E0FFD1851245AD90120FE0FF9026EF
:103AA00093E0FEEF4E90120FF0914DF14A7B017AB8
:103AB0002679961237C6500FC3902697E09420902F
:103AC0002696E0940340E6D185124B1212373E3021
:103AD0002E0221D5902698E0B40103D38001C322A1
:103AE000EB25E025E02401F582E43412F583E0FCC7
:103AF000A3E0FDA3E0FEA3E022902520121E28757E
:103B0000FF0243E180F115124FA3902535121E34B8
:103B1000002DC6C0E4F5FFF5A490120EF0A3F090BE
:103B200025307402F0D1C8FFF595EF1460181460C9
:103B3000262402703690252051EEFF902531121E6A
:103B40002890252C802090252451EEFF90253112BD
:103B50001E2890252D800F90252851EEFF902531AD
:103B6000121E2890252EE0902539F0124FCC90257A
:103B700039E0700FF5FFF56975FF0175D70975F428
:103B800018805990120EE004F0902530E0F1E39097
:103B9000253551EEFF902531F13FFBC3121DAF508B
:103BA0000A90253151EEFFA3121E28902539E0FF1F
:103BB000124E2490252FE0FFA3E0FDA22D922B12A0
:103BC0004F51A351EEFF902707121E28902530E099
:103BD000FFB1E4902530E051E1FFD18CD1D06002FB
:103BE00061257402F0D1C8F595E5F454077017907B
:103BF0002535916F7801121DC0902530D175121EA8
:103C00002851E0FFD18CD1D070DB75FF0375958012
:103C100090120EE0D39401400343F420A22D922C85
:103C2000124E8390253551EE2420FFEE344E9191B3
:103C3000E4FB7A04F9F8917F7801121DC0C22A12C0
:103C4000429BE4F5FFE5BD54F84404F5BD90121322
:103C50007401F07E127F01E4FDEF2DF582E43EF564
:103C600083E0FC901213E02CF00DEDB412EB22FF78
:103C70007E04FDFCE0F8A30EF9A3E0FAA3E0FB123A
:103C80001C77E47B7DFAF9F8121D02EF2401FFE4B2
:103C90003EFEE43DFDE43CFC229025F4F138E9F0E1
:103CA0009025FA121E34000000019025FE7401F0E8
:103CB000F5FFE5D554C070051237F15002C322E478
:103CC000F5FF53967F75FF0175D50412373775FFE1
:103CD0000143D508E4F5FF5394FBF5FF53847FF5CA
:103CE000FF7598FF9025F8E5F4F075F49C75FF01D9
:103CF000A3E5E4F075E4257B017A2579FED1E59012
:103D000025FEE064016002A1C2F5FF9025F774145E
:103D1000F09025FA51EEFF7801121DD39025FA128A
:103D20001E28E5A730E1FB43A7029025FA51EEFFDC
:103D3000E5A730E005E47B018002E4FBFAF9F8EF47
:103D40004BFFEE4AFEED49FDEC48FC9025FA121EB1
:103D5000289025F7E014F070B89025FA51EEFF781E
:103D600010121DC07B6D7A4E79C67841121C77EF18
:103D70002439FFEE34309119E4FBFA7901F8121D71
:103D800002EE547FFEE4FDFC1247849025FA51EECA
:103D9000FFEB6FFFEA6EFEE8CDEFCDCCEECCECFF93
:103DA0009025F4D1DCEF121B159025F4D1DC9000A6
:103DB00001ED121B2790120FE030E606E4F5FF75C7
:103DC000968075FF01E4F5D59025F8E0F5F475FFD0
:103DD00001A3E0F5E4124E729025FEE0B40103D396
:103DE0008001C322902706EFF0E4A3916F780112BF
:103DF0001DC0902706D175121E28901210E0FF6496
:103E0000806071EFC3947F5038EBD177C083C0825C
:103E100051EEFFEEC0E0EFC0E0901210E075F0044C
:103E2000A4AEF0FBCAEECAEA3395E0F9F8D0E0FFA1
:103E3000D0E0FEC3EF9BFFEE9AFEED99FDEC98807B
:103E40002B902706E0D177C083C082F13FFB901210
:103E500010E0F40475F004A4FFAEF0EE3395E0FD3D
:103E6000FCEB2FFFEA3EFEE93DFDE83CFCD082D0B2
:103E700083121E2822E0FB52E025E02401F582E4B3
:103E80003412F583227B017A267998229027371203
:103E90001E2875FF01902737A3E0FDA3A3E4FFFED2
:103EA000E4FC7810121DC08FE1902737A3A3E0FE39
:103EB000A3E4FFE4FDFC7808121DC08FE2902737D1
:103EC000A3A3A3E0FF8FE32275FF03902530E02238
:103ED000902530E0FF14F0EF22902744E0FBA3E0B0
:103EE000FAA3E0F922902763F138E9F07F017C1210
:103EF0007D01E4FEED2EF582E43CF583E02FFF0E1C
:103F0000EEB412F0901213E06F6009902763D1DCD9
:103F1000E4121B1522E5FA30E1FB75FC8075FF0108
:103F200053D5EFE4F5FC75FC40F131E5FC20E6FBF0
:103F30002275FF03E4F59122EBF0A3EAF0A322E05F
:103F4000F8A3E0F9A3E0FAA3E022E4F5FF75C2E1EB
:103F50007F1E12560A30E707E4F5FF75C2A122E47E
:103F6000F5FF75C28122902701EEF0A331C77FFFD4
:103F7000A3E0F9E9C3940C0523E9F19FE0FCA3E079
:103F80004C7016AF01902701E0FCF1CEA3E0902722
:103F900000F0124249E904FF220980D722E5617549
:103FA000F007A4242FF582E43424F58322F1EB50AA
:103FB0001412440CE0FCA3E0FD4C6009EFF19FEC0F
:103FC000F0A3EDF00EAF062275FF018FDA22A3E019
:103FD000FDA3E0FB2275FF0153D8EF22F1157F0806
:103FE000021AA733333354F8F5F422E4FE1FEFC36B
:103FF000940C229027057402F0E1669002B1E0640F
:10400000AA2411FFF022AE07123FFBEE04FEEF8E52
:10401000F084AFF02230260C902379E07006FF1276
:104020001A25C22611290219B23017241153FF9004
:104030000424E0FEEFC39E400AEF9ED3940240109A
:10404000C21722900424E0F42FD394014002C21737
:1040500022C2AD902483E0A3E0229002BAE0FCA348
:10406000E04C700A9002BAEEF0A3EFF0D322C32224
:104070009002BAE0FEA3E0FF4E6009CAEECAC9EFA3
:10408000C9121F2F22E4F557F558F559F55A75FF57
:104090000185FD5375FF0185C95475FF0185CA551A
:1040A00075FF0185CB5622EF11AEF0020000901291
:1040B00021F09027B922901221E0FFF460059027AB
:1040C000B9EFF074FF11AEE0FF22901221E0FE6420
:1040D000069027B96004EFF08008EEF0901221748A
:1040E000FFF09027B9E0FF22EFB40109D2AD75FFD0
:1040F0000143AE4022C2AD75FF0153AEBF2275C869
:104100000122E5C85402FF75C80222E5C85401FF28
:104110002275FF02D2ADD2BD75FF02758E71755F3B
:104120000975FF02E58E546F4480F58E22C0E0C011
:10413000F0C083C082C0D075D008C0FF75FF02E513
:104140008E30E42975FF02E58E54EF4410F58E9011
:104150000000E004F0E55F30E0020531E55F700B40
:10416000755F099024831227E48002155F75FF02B2
:10417000E58530E404318C5060D0FFD0D0D082D0BF
:1041800083D0F0D0E03275FF0253857F75FF024384
:10419000851022AB07AA063186ED4C70050DBD00D7
:1041A000010CD3ED94FFEC9403500AEDF586EC443A
:1041B00030F5858052D3ED94FCEC940F5017EDAEA2
:1041C000047802CEC313CE13D8F9AC06F586EC44BE
:1041D00034F5858032D3ED94F0EC943F5016ECC466
:1041E000F854F0C868FCEDC4540F48F586EC443828
:1041F000F5858013EDAE047806CEC313CE13D8F93F
:10420000F586EE443CF5859027935120D220E4F5C5
:104210006075FF0243854075FF02438580D21F22EF
:10422000AF03EAF0A3EFF0223186C21FE4F560C2CB
:104230002022301F0D3186E4F560D22075FF024345
:10424000858022E4F560C220229026FDECF0A3EDEB
:10425000F0AA07AF03EF70010FEF75F00AA4FFAEED
:10426000F0EA910DEEF0A3EFF0EA123F9FEEF0A31B
:10427000EFF0902700E0FFAE718DEFF09026FDE0AB
:10428000FEA3E0FFEA75F007A42433F582E43424AA
:104290005194F022F583EEF0A3EF2290253A121EFE
:1042A00028E4F5FF75BB0575BB8575FF0175D50263
:1042B000202A06123737123F4A75FF0143D52030B6
:1042C0002A026166E4F5FF538EF7438E077D04E40E
:1042D000F5FF8DBCF5FF43B102E5B130E2FBE4F53B
:1042E000FFAFDFEFFEACDEECFBEBFFED25E02438AB
:1042F000F582E434255194F0E4F5FFF5FF53B1FD68
:104300000DEDB40CCA90253A123AEEFF7809121D51
:10431000C0A3EEF0A3EFF0E4FDED25E02442F5822A
:10432000E43425F583E0C313FAA3E013FB7180F5B1
:1043300083E0C313FEA3E0132BFFEE3AFE7180511E
:1043400094F0ED240490120DF0EDC394075017CFB4
:10435000EDCF0DEF71819105FFC390253FE09F9058
:10436000253EE09E50B3E4F5FF758EC8F5FF901230
:104370000DE0F5BCE4F5FF57BB8075FF01F5D522D4
:10438000ED25E02440F582E4342522E56175F0074F
:10439000A42435F582E43424F58322900000E06003
:1043A00056E014F0E4F561E561C3940C50ED123F62
:1043B0009DE0FEA3E04E603B123F9D911B70347167
:1043C0008BE0FF6008F46005718BE014F0718BE006
:1043D0006011E561910DE0FEA3E0FF123F9DEEF05C
:1043E000A3EFF071F84E600871F8AA06F9121F2FBA
:1043F0001226A2056180B022E56175F007A424337E
:10440000F582E43424F583E0FEA3E022EF75F007A3
:10441000A42431F582E43424F5832274FFF5F012EC
:104420001BE645F022902302E0FF123FEB500F9174
:104430000CE4F0A3F0EF123F9FE4F0A3F00EAF0600
:1044400022121AADFF912AE4021B15902684121E37
:1044500091902684121E719141AE04AF0590268979
:10446000E0FDA3E0FB918E902684121E71EF121BDB
:10447000159026849184B4FF04E4121B15902684C1
:104480009184FF22121E71021AADE4FB7D01E490BB
:104490002705F0023F66A2AFE433FFC2AF9024834A
:1044A000E0FCA3E0FBAA04EF24FF92AFAE02AF034F
:1044B000221237F1500491C24003301703D3800118
:1044C000C322E5F754E024FF22AF14EFC36001D309
:1044D00022EFC3940E5005900415EFF022E5175417
:1044E0000FFF22E517C394F0501F5317F0B10CFED5
:1044F000740FC39F4005EE940E400543170D8003D3
:10450000EF4217E517540FFF227F0022E517C4542E
:104510000FFEEF9018E8932E22B10CFFC3940E40CB
:10452000027F0DEF9018CA93FF22EF30E303AF1321
:1045300022AD1B201804EE30E00BE517C394F050B9
:1045400020B17C8018E51A6006FDE4F51A8012E5BA
:1045500017C394F0500BE517540FFF6004B119AD69
:1045600007AF05224315015315DFB12AF13340048B
:10457000E4F514225315FB2135E9D322900415E00C
:10458000FDFFC3740EB1A6EFC4F8540FC868FFEE68
:10459000C454F048FEE51754F0C39FEE12339F7FDA
:1045A000005002AF05229FFFE49400FE2290273FB7
:1045B000EDF0901211E0FEF46006A3E0FDB4FF0CF4
:1045C0009027417418F0A37413F08008902741EEEF
:1045D000F0A3EDF0121AAD64016002E10D90273FE7
:1045E000E0FE64086004EEB404089027407428F0EC
:1045F0008006902740743AF0EF123AE1FF121DA1B5
:10460000E4F10EEF24D8FFEE343FFEED3493FDECE1
:104610003416FC7B007A807903780012184EF184FE
:10462000902742E0FF902741E0C3B1A6E4FCFD12D1
:104630001C77ECC0E0EDC0E0EEC0E0EFC0E09027FA
:1046400042E0FFE4FCFDFEF10ED0E0FBD0E0FAD04A
:10465000E0F9D0E0F8EB2FFBEA3EFAE93DF9E83C5F
:10466000F8902740E0FFE4FCFDFE121C77EF245495
:10467000FFEE340B123C914E7BA87A16F9F8121813
:104680004ECBEFCB90273FE014605D14601B24FEFF
:10469000600C24FC7077E4F5FF75CE318006E4F5FC
:1046A000FF75CE21F5FF8BCF22E4FAE4F5FFEA2473
:1046B00040F5CEE4F5FFEAFFC37407B1A674F72F07
:1046C000F58274183EF583E4F116C39DF5CFE4F549
:1046D000FFEA2448F5CEE4F5FFEA9018F7F1162D2D
:1046E000F5CF0AEAB408C422E4F5FF75CE01F5FF60
:1046F0008BCFF5FF75CE0EF5FFEB25E0F5CFE4F59A
:10470000FF75CE0FF5FFEB75F003A4F5CF227B64A8
:10471000FAF9F8021C779325E0FDE433FCEB75F021
:1047200010A4FFAEF0121B5BCDEFCDEBFFE4C31383
:10473000EF1322900437EFF0900414E024FD601191
:10474000047007F17A7404F08012F17A7408F08032
:104750000BE4900438F09004367402F07F01121AD2
:10476000A7900438E0FF900436E0FDA3E0FBE4905E
:104770002695F01239D0509ED3229004387401F05F
:1047800090043622C8ECC8C9EDC9CAEECACBEFCB3B
:1047900022E51754F0C4540F2FFFC3941040027F3A
:1047A0000FEF9018D893FF227E10EE60091EEE9056
:1047B00018D893B507F4EEC3940E40027E0DEE9028
:1047C00018CA93FF22E4F514E514702712561C1240
:1047D00037F15005C22F1233BE123FDC12361EE5F0
:1047E000D120E0FB4315205315FEE4F510A21692EC
:1047F000EDD322C322C2AFEF4215D2AF22EF24FE87
:10480000600C24FE600580007F01227F02227F036E
:1048100022E51520E50812361AE5D120E0FBE4F583
:104820001022301704C217112A22C221E4902766F1
:10483000F0C222A3F0A3F075FF01E5D520E702C383
:1048400022C23011F420210201E053F4DF902766E8
:10485000E0FF12362A75FF0143D81030220543F4D9
:1048600040800353F4BFE4F5FF53F5F0902767E071
:10487000FAA3E0FBEA42F5BEF5F6D23011F47FC8A8
:1048800012370BE4F5FFE59320E6051237A240F35B
:1048900030225FE5F430E3047D288010E5F430E257
:1048A000047D288007E5F430E1027D28123F317F46
:1048B0002812370B1237A240FB7F7812370B1237C2
:1048C000A2502F31A650F731CDEFC39D50F031A645
:1048D00050ECE5F720E5E7C23011F4123F3180DEFD
:1048E00053F4BF90120EE0D39401400643F420121B
:1048F0003FD5D322AFF4EF547FF5F4303005EF44C9
:1049000080F5F475FF01E5D520E702C322E5F4D375
:1049100030E601C322900445EFF0C23011F4D221F9
:10492000900445E0902766F0D222A3E4F0A3740D32
:10493000F01137E4900446F01237F15038900446F5
:10494000E07032E5F754C060EF318B319EBF5511F6
:10495000319E90121CE06F90044670147402F08037
:10496000D7900446E0B454057433F080CB900446ED
:104970007401F080C3900464E0B40207C22F1233C4
:10498000BE8000112A900446E0FF22E5F720E008EF
:10499000E5F754C070F5FF2243F701AFF922318BE0
:1049A000900446EFF02275FF01E5E43322E4FFE5D1
:1049B000F754C06002801675FF01E5D530E30D3174
:1049C000A650F431CDEF60EF31A650EB227108AF65
:1049D000D9225315FEE51530E5057F0112362A511F
:1049E0002EEF70FB7F02121AA77F01311590044C45
:1049F000EFF0BF0202801390044CE0B43311E4F0F6
:104A00007F013115BF020D90044C7401F08005E464
:104A100090044CF090044CE0700D1237F15005C238
:104A20002F1233BE123FDC90044CE024FF22E490AE
:104A3000273BF0A304F0E490273EF0E5FA30E1FBD9
:104A400075FF01E5D530E7037F0022E4F5FF75E54A
:104A500008123FD5E5D530E61A75FF0190273DE5F0
:104A6000DAF0E4F5DA75FF01E5D630E3FB90273E96
:104A70007401F075FF0375B90475FC4175FF03E51A
:104A80009B30E7FBE4FB75FF038B95123AE0FF12C6
:104A90003E8C0BEBB403EF75FF03759580E4F5FFD7
:104AA000758EC8123F4A75FF0153D5FB123F317F07
:104AB0001412370B12373E75FF0143D50490273E81
:104AC000E0700B123F317FC812370B12373E7B016B
:104AD0007A27793C711290273CE090273B7006E0E2
:104AE0004404FF8002E0FF90273BEFF090120EE0BD
:104AF000B4010675FF0143D81075FF0190273DE012
:104B0000F5DA90273BE0FF2275FF01E4F5EA75EA4C
:104B1000FF22C22975FF03759B1F75FF0390120FBB
:104B2000E0FF20E71BE59A540FC394024012EF44C4
:104B300080F0E4F5FF75C2A143FC0475FF03D229A0
:104B4000E5FC30E609E59A540FC3940540CCE5FC3A
:104B500030E611E4121B1575FC80F5FC75FC40E590
:104B6000FC20E6FB302903123C4D22900425E0A3F3
:104B7000E0FF22900442EF0FED24FE60191460263E
:104B80002402703BEB2402FFE43AFE7C007D5012CD
:104B90001B497D60801E71E7C333CE33CED8F9FF49
:104BA0007C007D28800E71E7C333CE33CED8F9FF69
:104BB0007C007D64121B5B900443EEF0A3EFF09049
:104BC0000442E071F2C083C082121E1C900444E0D3
:104BD0002401FF900443E03400FEE4FCFD121C5C61
:104BE000D082D083021E28EB2401FFE43AFEEF7846
:104BF000032225E025E02418F582E43404F583221D
:104C0000EF71F2121E00021DE6E49004189120E4F8
:104C100090041C9127E4FFFEFDFC900420021E2856
:104C2000FFFEFDFC021E28FFFEFDFC021E28E4FF25
:104C300075F0E5EF900001121E65E4F00FEFB4038C
:104C4000EFE4F56222900447EF91BBFEFD75F0E5BD
:104C5000ED1227F5FC700C900448E0B4FF02EDF073
:104C60000F8006EC30E0027E010DEDB403DF90040E
:104C700047E06401600DEF3C94025007EE7004A31E
:104C800074FFF0900448E0FFC39403501FEF122F0D
:104C9000107DE5E4FF121958900447E04410FFA38B
:104CA000E0FE75F0E591B3F0EE022F107B007A0084
:104CB000790022900001121E65EF22F0A374FFF02C
:104CC000E4FF22E4021B15121AAD540F021B1580DB
:104CD000F6EF7011ED600775FF0143AE012275FF1D
:104CE0000153AEFE22EFB40110ED600775FF0143E2
:104CF000AE022275FF0153AEFD2275FF02E5E630DC
:104D0000E2037F0322E5E630E3037F0022E5E6309D
:104D1000E1037F0422E5E67F0530E0027F0122EF18
:104D2000600775FF0253E6BF2275FF0243E640228B
:104D3000EF14600F146014240270188B8075FF014B
:104D40008DFD228B9075FF018DC9228BA075FF010F
:104D50008DCA22AF038FB075FF01AF058FCB2290B4
:104D6000268C121E91EF14601414601E240270270A
:104D7000B1A5E580B1AB12E171E5FD8025B1A5E5F6
:104D800090B1AB121E71E5C98018B1A5E5A0B1AB19
:104D9000121E71E5CA800BB1A5E5B0B1AB121E7150
:104DA000E5CB021B1590268F021E71121B1575FF95
:104DB0000190268C22E4F5FFAF9122E4F5FFAF923B
:104DC00022E4F5FF75D102E5D120E0FBE4F5D1F551
:104DD000FFEFB1E2EE540F42D6E4F5FFCFEDCF8FF7
:104DE000D422F5D7E4F5FF53D6F022E4F5FFEFF532
:104DF000D8E4F5FF53D60FEE540FC4F854F0C8E4CE
:104E0000C4540F4842D622E4F5FF8FD422E4F5FFC4
:104E1000E5D1540133333354F8FFE4F5FFE5D354BF
:104E2000074FFF22EF30E00E43F401E4F5FF43A407
:104E300004F5FF759624EF30E10E43F401E4F5FF2D
:104E400043A408F5FF759624EF30E20943F402E429
:104E5000F5FF75961EEF30E30943F404E4F5FF75A2
:104E6000961075FF01EF5403600475D7122275D7B1
:104E70002D22E4F5FF75846EF5FF439404F5FF756C
:104E8000981422E4F5FF75933F75FF03759A40D19E
:104E900072E4F5FF759C93F5FF75A1A3F5FF758589
:104EA00031F5FF758628E5FA54304480F5FA75FF30
:104EB0000175E74A75FF0275DF4975FF0143D304A9
:104EC00075FF0153D367E4F5FF53E6BF75FF017526
:104ED000D825F5FF75B503F5FF75B215F5FF75BA61
:104EE00002F5FF75AFB3F5FF75CD0AF5FF75CB0879
:104EF000F5FF75CA12F5FF75BF0EF5FF75CC96F577
:104F0000FFF5BDF5FF75C281F5FF75AEE1F5FF75E3
:104F1000DA55F5FF75F580F5FF75E903F5FF75E9DD
:104F200033F5FF75972A75FF01759B42759CA47533
:104F30009D29759E48759F2475A11275A312759AB7
:104F4000F8202C0CF5FF43968090120FE04440F0BF
:104F500022CCEFCCCFEDCF74017E00C8EFC8088023
:104F600005C333CE33CED8F9FFCDECCDEF5D601B5A
:104F7000302B1875FF0175CDAD75FF0175DDCDE4E2
:104F8000F5FF759A74F5FF7594842275FF0175DC41
:104F90005375FF0175DD33E4F5FF759A14F5FF7560
:104FA000940422F1C253DB7F75FF0175D5027F1493
:104FB00012370B12373EF1C243DB8075FF01E4F577
:104FC000D52275FF01438E1075FF012275FF017513
:104FD000E46575FF0175D6472275FF01E5D530E61A
:104FE00002C32253FACFEFB4080543FA308012EF20
:104FF000B4040543FA208009EFB4020543FA108097
:1050000000D322E5F45418131313541FFF22E5F7BD
:105010005406FFBF06037F0822E5F75406FFBF04CE
:10502000037F0422E5F75406FFBF02037F02227FBD
:10503000012275FF01E5D520E602C322E5FA5403FB
:1050400060FA75FF018FC3D322CEEFCE75FF01E565
:10505000D520E602C32243FA04E4FDEDC39E5007C7
:105060007F5511320D80F4E5FA543070047F0F80C3
:10507000027FF01132D3225EF71322E5F754C024E9
:10508000FF22E490251FF07B017A2579061227FD87
:10509000902508E0FBB4112290251B121E3400005D
:1050A0007800902517121E34000060009024FC74D4
:1050B00018F0A3E4F0A3F0A380277412D39B502729
:1050C00090251B121E3400020000902517121E347A
:1050D00000020000E49024FCF0A3F0A37418F0A3F5
:1050E000E4F090251F04F090251FE0FB6017E4FF1B
:1050F000FE7D02FC902508E024EFF9F8121DD39004
:105100002500121E28AF03229027B3EFF0E4A3F08E
:1051100090251FE06029E4FFFE7D029025003145C7
:10512000700851477E777D00800A71EB501151471E
:105130007EFF7D017C00122496E4339027B4F0902A
:1051400027B4E0FF22FC121E1CC3021DAF902628CC
:10515000121E9190262BECF0A3EDF090251FE0702D
:1051600002411AE4FFFE7D02FC9025003146704C9E
:105170005134314650465125A3512EE4FB7A18F99B
:10518000F8C3121DAF503590262D121E1CC3E49B90
:10519000FF74189AFEE499FDE498FCE49026298FA8
:1051A000F0121BE6C390262CE09FF090262BE09493
:1051B00000F090262D121E3400001800513D512E93
:1051C000A804A905AA06AB075152121C5C90250041
:1051D00071FB404171EB4023E4513431464036903D
:1051E000262BE0FEA3E0FBE49BFF74A09EFE74016F
:1051F0009400FDE49400A33145501A513D512EC056
:1052000007902628121E7190262B9111D00712307C
:1052100004E4338001E4902631F0902631E0FF224F
:105220009024FEE0FEA3E0FFE4FCFD90251B121E8F
:105230001C021C5CFF7E18FDFC90262D2290262D62
:10524000121E00902517229027B3E09026FBF07FD6
:10525000FF2290262BE0FEA3E0FFE4FCFD22902736
:1052600090121E915120EF2408123C8E7B017A256A
:10527000790471B97402F0212614902504515590D7
:105280002517512E7B017A25790971B9740EF01218
:10529000261471C0EE3480123C9171AC90250B71D4
:1052A000CA7F0F7E1D719871B2C006C00771C0E43D
:1052B0003E71D771AC90250D71CAD007D006719898
:1052C00071B2C006C00771C0EE348071D771AC9066
:1052D000250F71CAD007D006719871B2C006C007F9
:1052E000512071AC90250AE02400FE902509E0349D
:1052F000E890248BF0A3CEF0D007D0067198121C52
:105300001245F0C37001D322902485EEF0A3EFF094
:10531000A3121E0090248D121E2890248BE0FFA360
:10532000E0902491CF8062902491E0FEA3E0FF4EB4
:10533000605DC3EF9440EE94004006A37440F0809B
:1053400005902493EFF071E0FF71B9EFF090248D98
:10535000121E00122614902493E0FFC3902492E0C2
:105360009FF0902491E09400F090248D121E1C90E8
:105370002493910290248D211E28718F71E0910950
:10538000EDF01219D0902485EEF0A3EFF080989004
:105390002485E0FEA3E0FF227108902790121E7181
:1053A000EE8FF0121C3D902790021E719024870210
:1053B0001E28121C12FFAEF022902642E4F0A32217
:1053C000902517121E00E42FFF22E0FFA3E0902497
:1053D0008BCFF0A3EFF022FEED3401FDE43CFC2284
:1053E0007B017A247994902493E022902500121E68
:1053F00000E4FBFA7904F8D3021DAF121E1CD3029D
:105400001DAFE4FCFDFE021C5CFD90266BE4F0A3E6
:1054100022E0FFA3E09025F0CFF0A3EFF022EF60B1
:105420000A75F28075F24043F14022E5F130E7065B
:1054300053F17F43F180E5F130E308E5F230E7FB1B
:1054400075F2C022E5F130E70653F17F43F1802287
:10545000EF600443F1802275FF01E4F58E53F17F84
:1054600022EFB4080C75FF01E58454FC4403F58475
:1054700022EFB4040C75FF10E58454FC4402F5845B
:1054800022EFB4020C75FF01E58454FC4401F5845D
:1054900022EFB4010675FF015384FC22E5F130E4EC
:1054A0000F75FF0175FF015385F075FF018F86228F
:1054B00075FF01EF540FFDE58554F04DF58575FF3F
:1054C00001EEC4F854F0C8EFC4540F48F58622EF3B
:1054D0006003D2EA22C2EA2275F24022E5F2C3302A
:1054E000E601D322E4F55DF55EE5F230E72675F2DC
:1054F00080E5F1AFF330E407755D008F5E8010EF5B
:1055000075F010A4F55E85F05DE5F2540F425EAED5
:105510005DAF5E227EFF7FFF22EF600775FF0143D4
:1055200084042275FF015384FB2275FF0153853FDC
:10553000EF428522EFB4010443F1102253F1EF2230
:10554000EFB4010443F1042253F1FB22EF60044362
:10555000F1012253F1FE22EFB4020343F108EFB44C
:10556000010353F1F7EFB4030543F101803FEDB4BC
:10557000040875FF014385028014EDB40107B1B141
:105580005384F78009EDB40205B1B1438408EBB44C
:10559000100875FF015385EF800AEBB4200675FFF4
:1055A0000143851075FF01902762E0F58E43F1807D
:1055B0002275FF015385DF75FF0122121E71E92458
:1055C00001F9E43AFA22EEF0A3EFF0A3021E917B78
:1055D000017A12791C9026C5121E917A0222E0FCF3
:1055E000A3E0FDD39FEC9E22A3F0E4A3F0A322F05E
:1055F000A3F0A3F0A322E5122407F582E4351122DB
:10560000E4F5FFE5D25480440A22FE1236C9901216
:105610000FE022E5D254804414F5D222C2EBA2ED71
:105620009216C2ED22FFFFFFFFFFFFFFFFFFFFFF0C
:10563000FFFFFFFFFFFFFFFFFFFFFFFFFFFFFFFF7A
:10564000FFFFFFFFFFFFFFFFFFFFFFFFFFFFFFFF6A
:10565000FFFFFFFFFFFFFFFFFFFFFFFFFFFFFFFF5A
:10566000FFFFFFFFFFFFFFFFFFFFFFFFFFFFFFFF4A
:107FB000FFFFFFFFFFFFFFFF7FC607F9318C0001C6
:107FC000001E010A7AA4FFFFFFFFFFFFFFFFFFFF74
:107FD000FFFFFFFFFFFFFFFFFFFFFFFFFFFFFFFFB1
:107FE000FFFFFFFFFFFFFFFFFFFFFFFFFFFFFFFFA1
:107FF000FFFFFFFFFFFFFFFFFFFFFFFFFFFFFFFF91
:108000007B01E4FF902769121E91AE051DEE601002
:10801000902769E475F001121E7AEF121B1580EAB1
:1080200022712A4AC36001D340026118E924B77162
:1080300022FF7B017A2779BF12BFD930010B712A49
:108040002402712230E50221AD712A24B67122FF8B
:1080500090121CE06F703B712A24B7712230E73216
:10806000712A128801128FF9540764037024712A4F
:1080700024B97122D394400519712A12880112BAC9
:108080000312BF9944047132712A24BB7122441037
:1080900021A8712A24B7712230E721540F6401709E
:1080A0001B121AAD30E70F712A24BB712230E4068F
:1080B0007E007F0180117E007F00800B712A24B733
:1080C00071225410FF7E00EF4E601A712A24037152
:1080D0002254FB121B15712A128801121C1254F82B
:1080E0004403129F9E712A2402712220E20221ADD4
:1080F000712A24DF7122D39403400221AD712A2416
:10810000037122FF30E431712A12B74EEF54EF129F
:108110001B15712A2406F9E43AFA128FF9712A1212
:10812000880112BA09EF54076402C37001D312BB6D
:108130007E9027BFE04F610B712A24DF7122D39418
:1081400002500C712A24BA7122FF12AF54801C9085
:108150002015E09021046008E004FF12ADD78006EE
:10816000E004FF12AE93902104EFF0712A128F67A2
:108170007403121B15902140E0F460071288085028
:1081800002610D712A24DF7122C39404501F712AE9
:10819000128801128FE67001D312BB7EEF44017189
:1081A00032712A128F677404121B15610D3001029F
:1081B0006113712A24DF7122C39405400261137197
:1081C0002A2403712220E0026113712A24B671224D
:1081D000FFC007712A24BA7122FD712A12BF4EC056
:1081E00003C002C001712A24B17122902652F0719D
:1081F0002A2402712254034401902653F0712A125A
:108200009DB5121C12FF902654E5F0F0A3EFF0D0BC
:1082100001D002D003D0071288D7EF700261131289
:1082200089B3240571224420FF1289B324141288D3
:10823000CF1289B312BF7E1289B012BFA111049070
:108240002283121E717405121B1590228312334370
:1082500012BF6E712A12BF59712A129DB5741A7518
:10826000F02A121C3D712A128801121C12AEF05421
:10827000F812BA08EF12BA601289B324047122FF0F
:10828000712A24021288CF1289B324067122FF7446
:1082900040C39F5008712AF1F1742F80167411D3D6
:1082A0009F500BEF24EFFF712AF1F1EF8005712A47
:1082B000F1F1E4121B15712A24B17122FF712A1207
:1082C000BF4EC003C002C0011289B3241C128F32FA
:1082D000D001D002D003128F42712A128FBF7B01CE
:1082E000C003C002C0011289B3128FD67B01128F66
:1082F00036D001D002D0037F11128F42712A128F23
:10830000677405121B1512BF9944067132129F8AB9
:10831000024CC7E4FF1298DB22902614121E71E96A
:108320002407F9E43AFA021AADFE9026E1121E7112
:10833000E922FF9026E1121E7190270B121E91EF89
:10834000540FFEF14624B8712254F0FDEF54F0FFB3
:10835000C4540F4D121B15EE14605F147002C13C23
:1083600024FE7002817824FE7002C1A824036002FA
:10837000E12FF146128FBF0C03C002C001129F8093
:10838000128F36D001D002D0037F04128FEFF14656
:1083900024B6F9E43AFAEFF14312C6D97403F14373
:1083A00024B8712254F012BF764FF14312D0E47416
:1083B0000AF14312C6E07409E12C128F6EF14612E5
:1083C000C6D97401F1432402712230E02320E70270
:1083D000800A90210EE0540FFFBF0F0BF14624B727
:1083E00071224440121B15F1461255BF74038007D9
:1083F000F1461255BF7401121B15F1462402712279
:1084000030E10BF14624B771224420121B15F146CE
:108410002403712230E20BF14624B771224410127A
:108420001B15F1462402712230E70BF14624B77187
:10843000224480121B1590121DE0FF7E0030E502E1
:108440007E20EF7F0030E4027F40EF4EFFF14624B4
:10845000B87122549FFEEF54604EF14324BA71224A
:10846000FFF14624D91288CF7F09F14624B1712249
:10847000F13012C6E0EFE1C2F1462402712220E69B
:1084800002A116F1462409712212D10E90270FF095
:108490007404C39E500B7404F0EF540F4440121B3D
:1084A0001590270FE02402FFF14612C6E7C003C073
:1084B00002C001F1462408128F32D001D002D0034D
:1084C000128F42F14624B17122FF90270FE024035E
:1084D000FDE43312339A4036121AADFF90270FE0B5
:1084E000FE2403FDC3EF9DFFF14312BF4EC003C046
:1084F00002C001EE240AFDE433FCF1462DF9EA3C0A
:10850000128F35D001D002D003128F428008F1467D
:10851000F1F1E4121B15128F6EF14612C6D97401E7
:10852000121B154480F1432402712290270B30E086
:10853000071255BB740380051255BB7401121B153D
:10854000F14612C6E7E4F1432403712230E20BF155
:108550004624BB71224410121B15F14612880112E9
:108560001C1254607002A1EEF14624B67122FF90F5
:10857000121CE06F7078F16424BB7122FF20E06E62
:10858000F1462403712220E465F14612C6E7EF4468
:1085900008F14324BC712290270B12D04124BD1254
:1085A000C101E4F14324BC7122C4540FFFF14624FD
:1085B000BD12C101121AAD4410F143128801121C00
:1085C000125460FFF14624BC7122C4540FFD7C009C
:1085D000F1462DF9EC3AFAE924BEF9E43AFAEFF162
:1085E00043128801121C12549F129F9E800BF14669
:1085F00024BB712254F7121B15F14624BB712230A3
:10860000E31DF14624BC7122C4540FFF7E00F146E5
:1086100024BD12C101121AADC4540F04FF80027FA1
:1086200000F14624BC7122C4540F240B2FFFF146E5
:1086300024B17122F13012C6E0EFE12C128F6EF1FD
:108640004612C6D97402F1432402712230E10BF1C3
:108650004624B771224420121B15F14624BAF9E4CE
:108660003AFA741DF14312C6E7C003C002C001907C
:10867000200A121E71128F63D001D002D0037F1D19
:10868000128F42F1461255BF7401121B157F26F15D
:108690004612C6E0EFF14324B17122FEEF042EFF33
:1086A000F14612D0E4EFE12CF14624B87122540FC8
:1086B00090270EF0F1462402712220E642128F6EBE
:1086C000F14612C6D97405F1432402712230E10B40
:1086D000F14624B771224420121B15F14624B871CB
:1086E0002254F0FF90270EE04FF143240271223014
:1086F000E016F14624B771224440121B158009F19F
:1087000046F1F174FF121AF3F1461255BF7401F1EC
:108710004312C6E07411F14324B17122FFF14624E3
:10872000D871222F04FFF14612D0E4EF121B15225C
:10873000FEEF042EFE90270B121E71E924B9F9E416
:108740003AFAEE121B1590270B121E71E9229026A1
:10875000E1121E91E924017122D39401403912B82B
:10876000B99026E5EFF07E1A7F4D712A24B7712269
:1087700030E719712A24BB172220E010712A24BC8B
:10878000712212D0F4B504047D07803F712A24B110
:10879000712212D1068034E49026E5F07E1A7F4DD6
:1087A000712A24B7712230E719712A24BB71222063
:1087B000E010712A24BC712212D0F4B504047D07A4
:1087C0008009712A24B1712212D1067C0090279B66
:1087D000EEF0A3EFF09026E07401F0AE04AF0512C6
:1087E000B7FCAC06AD0790279BE0FEA3E0FF02417B
:1087F0009324B1F9E43AFA2201FF90255A121E712E
:10880000E92404F9E43AFA22902104E0F470020128
:10881000C67880E6FF12832A24BA11CF12832A1168
:1088200001121C125418FD12BFAC12832A1101E46C
:108830008FF0121C3D121C12FFEF4D129F9E78818B
:10884000E6540F90279EF06038E0FF7404C39F4009
:108850003090279D7404F012832AF1C6C003C00231
:10886000C0017B007A007982F136D001D002D003BA
:10887000F14290279EE09062E1F1DD24BC11CF80AF
:108880000690279D7401F090279DE064047011E02C
:108890001283291101F1E67001D39223D2248012B0
:1088A00090279DE01283291101F1E67001D39223F4
:1088B000C22412BB82EE4F90279DF0D20390279DD9
:1088C000E0128332D322C322FF121E71E92408F979
:1088D000E43AFAEF021B1590264DEFF0A3EDF0A35A
:1088E000121E91902652E0D3942F400221AD12CD5A
:1088F0005D8F32EFC39402400221ADEF12D061745C
:108900000131B01255BFE4121B1590264DE0FF3126
:10891000B3240F11CFFF31B3240211CF90264EE0C4
:10892000FF31B3241311CFFF31B3240311CF9026AD
:1089300053E012D10E31B32405F9E43AFAEE121BDA
:1089400015EF540FFF31B3240411CF902652E0FFEE
:10895000602990264F121E71EA494B601E31B324E4
:108960001CF9E43AFAC003C002C00190264F121E5F
:1089700071F136D001D0020D03F14231B32416F962
:10898000E43AFA74FA121B15902652E02411FF31D2
:10899000B3240611CF902654E0FEA3E0FF31B324A8
:1089A00009F9E43AFA12BA09E53204FF227F0022FB
:1089B000121B15902283121E71E92290275B121E52
:1089C00091121E9AE92409128322541FF535B156DB
:1089D00012831FFFE5306401601C7412D39F501690
:1089E000E535B402067419D39F500BE535B4010880
:1089F000741DD39F4002C322B156E9240A12832278
:108A000030E21CB156E92408128322FF90121CE0C8
:108A10006F600CB156E92404128322FF12A22BE5E9
:108A2000356402600241DB90275B12831C30E70251
:108A300041D9B156E92408128322FF90121CE06F3D
:108A4000702A20140241D9C214B156E924041283B9
:108A500022FD7F0312CC04B156E92404128322FFC5
:108A6000D231B156E9241312A8A0806DB156E92481
:108A70000C128322FF540FEF605FB156E9240DF909
:108A8000E43AFA1E7C00E92E129F5EFD90121CE073
:108A90006D7046B15612831F6419703DB156E924BA
:108AA0000CF9E43AFAEF54F024102E121B15B156CB
:108AB000F1D5E4121B15B156F1367F18F13CC20313
:108AC000B156E92404128322FFB156E92408128327
:108AD00022FD12D04CF012BBDBC322E4FFB156E9F9
:108AE000240D12D0FD129F5EFE90121CE0B506020E
:108AF000C3220FEFB404E6B156E92404128322FF27
:108B0000B156E92406128322540FFD12CCB4500250
:108B1000C322B156E92408128322FF90121CE06F91
:108B20007002816F90121DE0FF54306002816FEF80
:108B300020E002816FE5356401600990275B1283B4
:108B40001C30E71F201302816FE53564016002814C
:108B50006FB156E92411F9E43AFEAF0112A7EE40D5
:108B600002816F12CD5D8F32BF0202C322B1561255
:108B7000831FFF7440C39F0502C322E535B4011D66
:108B8000B156E92411F9E43AFA7B01C002C0017A36
:108B90000279B6F136D001D0027F04F142E53212FB
:108BA000D061B15612831FFF31B3F1D6C003C002AA
:108BB000C001B156F136D001D002D003F142B15616
:108BC000E92404128322FF12CCFFB156E9240612D5
:108BD0008322540FFE12CCF6A606F1CDF8760708D4
:108BE00076D0B156E9240C12832254F090275EF01F
:108BF000607DE0FF7440C39F4075E024F0F031B326
:108C00002417128322540FFF7404D39F40619012E3
:108C10001CE0FE31B3241812D0FDF9EC3AFAEE1242
:108C20001B1590275EE02F04FF31B3241711CFB13D
:108C300056E92404128322FF31B3240211CFB15626
:108C4000E92408128322FF31B3240311CF90228339
:108C500012CA119022831287FD7440121B15B1565F
:108C600012831FFF31B3240611CF31B312D0BEB12E
:108C700056E92408128322FF90121CE06F6006EF71
:108C8000F46002A15290275B12831C30E702A152CC
:108C9000E5356002A152B156E92411F9E43AFAC06F
:108CA00003C002C00190275B12B74A121EBAB15628
:108CB00012831F24EEFF90275B12BF4211CF902733
:108CC0005B12831C4401121B15B156E92405128363
:108CD0002230E677B156E92404128322FFC231B173
:108CE00056E9240C12A8A0B156F1367F11F13C9040
:108CF000228BE054BFF0B156E92404128322902263
:108D000097F0B156E92406128322540F902298F06E
:108D1000B156E9240CF1327B017A2279997F05F171
:108D2000EF90228AF090228D7419F0B156E9240454
:108D3000128322FD90228EF0A37422F0A37407F018
:108D4000C20312D04CF012BBDB8009E535C37001C1
:108D5000D322C322D32290275B121E71021E9A9047
:108D60002552EBF090255D7401F090255FEFF090B7
:108D70002557E0FE54C070C3902556E0FCD3949F65
:108D800040037F0022902552E0B4FF09ECD39436D3
:108D900040037F002230060C902556E0D3942E40ED
:108DA000037F0022EE20E40C902556E0D3949740F8
:108DB000037F0022F12724B6F9E43AFAED121B15DD
:108DC000902552E0F12624BA11CFF127F167E41281
:108DD0001B1530060CC20690255A12B74A74018042
:108DE0000F902557E030E60BF1B4F127F1677405D9
:108DF000121B15902557E05490705A90255DE06441
:108E000001705290255A121E7112B8DEEF604612A0
:108E100087FA121C125460600E90255A12B68B12FB
:108E200083224410121B15F12724BC12832254F014
:108E30006002F1B4F127F1677402121B1590255FEF
:108E4000E05498F0E0FF1287FA121C125467FEEF0C
:108E50004E90255FF0902552E0FDB4FF0790255716
:108E6000E054FAF0F12724DF128322707090255726
:108E7000E0540564057066FA0512AF54505812BFED
:108E8000AC90255FEFF07881E6540F90255EF0609E
:108E900031E0FF7404C39F4029F127F1C6C003C02D
:108EA00002C0017B007A007982F136D001D002D075
:108EB00003F14290255EE090255AF1DD24BC11CFEC
:108EC000F1B4F127F1677403121B157880E6F126DF
:108ED00024BA11CF8007902557E054FBF0F12724E6
:108EE000DF12832270057404121B1590255FE0FFCA
:108EF00090255DE0FD902556E09025AFF090255738
:108F0000E09025B0F0902558E0FBA3E09025B1CB90
:108F1000F0A3EBF090255A12C48A902553121E71CB
:108F200012BA0F7F0122FF90255A121E71E922E921
:108F30002403F9E43AFA9026A4021E917B017A22D6
:108F400079869026A1121E91AE071FEE601890261A
:108F5000A4E4122749FE9026A1E475F001121E7ABE
:108F6000EE121B1580E22224DFF9E43AFA22902760
:108F70000B121E71902775211E9190277530051DCB
:108F8000F1BBC003C002C0017B017A2179B4F13684
:108F9000D001D002D0037F04F142C20522F1BBC050
:108FA00003C002C001129F80F136D001D002D0036D
:108FB0007F04808E90255D7404F022121E71E924D6
:108FC000B2F9E43AFA2224BDF9E43AFA22EF25E0B4
:108FD00025E0243822E9240BF9E43AFA22C454F0BB
:108FE000FF121E71E922121C1254076402C322F1FF
:108FF0004290121CE0FF221100121C12FFAEF02260
:109000000224579026C2121E9112CA0A9026C51237
:109010001E71EF121B159026C2121E71E94A600CD8
:109020009026C2129F9712D02712275C22902614F6
:10903000121E91121E9A90261B121E919026141237
:109040003343E4121B15C204902016F012D0D7123D
:109050008F367B017A2079047F04128F42202713F8
:10906000129F8012A83C12A7E46008128319448062
:10907000121B15128319307E6A90121CE060333087
:109080001330F1B02405128322540FFF640560539E
:10909000EF6401701D121AAD30E717F1B0240A1207
:1090A0008322F1AA12C0FF12B74D129F7A12A7E8CD
:1090B0006031200E02C1E7201029F1B0240512838F
:1090C0002220E71FF1B012D0752401128322B403CD
:1090D00012F1B02409F9E43AFA12B74D12A7DC7084
:1090E00002C1E7F1B02406128322540FFF90200240
:1090F000E07E00B402027E80EF4E9021B3F0128336
:109100002A4A604AE924B7128322FF7B017A267932
:109110001712BFD912832A128801121C125407FF9A
:1091200012832A24B8128322540FFE902617E0548B
:109130000FFDBD04047D4080027D00EE4DFEEF7FFB
:1091400000B402027F80EE4F902009F0800690204C
:109150000974FFF0F1B02405128322FF540F24FE9E
:109160007002C113147002C1B524FE7002C1DC2468
:10917000046002C1E79026B112831CFE740AD39EDC
:1091800040028029EF20E702A1B39021B3E04440E0
:10919000F0F1B0240A128322C4540F902618F06014
:1091A0000CE0FFD394045005740B9E400A902614E3
:1091B000123343E4021B15F1B0240912832230E17B
:1091C0002630E32390261B12831CFDEF240DFFE4C1
:1091D00033FEC3ED9FEE12339F500CF1B024091201
:1091E000832254F7121B15F1B02409128322902612
:1091F0001B30E35012D0DD128322F1AA12C0FF12FD
:109200001AADFFC4540F29F9EE3AFA1255BEC00345
:10921000C002C00112B747121EBAF1B0240A12836D
:1092200022C4540FFFFD7C00F1B0240BF9E43A1284
:109230009F5BC4540FFE90261B12831CC39FC39ECA
:1092400024F3802C12D0DD128322F1AA12C0FFC0B9
:1092500003C002C00112B747121EBAF1B0240A12AD
:109260008322C4540FFF90261B12831C24F4C39F37
:1092700012BF3E1288CFF10B2408128322FF9012F6
:109280001CE06F6002619EF1B0240A128322540F29
:10929000FF902618E06F6002612F902003E06002CB
:1092A000A114F1B0240512832290261430E607128F
:1092B000831C440D800512831C4409121B15F1B058
:1092C000128FD67E0012C105E924FFF9EA34FFFAB5
:1092D000121AAD9026141288C812831930E702A121
:1092E00014F1B0240512832220E702A114F1B02466
:1092F0000A128322C4540FFFF1B012C0FF121AAD3C
:10930000D394014002A114E9240112832264036072
:1093100002A114F1B0240A128322C4540FFFF1B049
:1093200012C0FF128F2F7B0112D0EBD205A114F1D6
:10933000B0240A128322540F640F6002A114F1B00A
:10934000240512832230E6081283194404121B15E7
:1093500012C26A501BF1B0240A128322C4540FFFB8
:1093600012D0D712C08B50081283194401121B155A
:10937000F1B02409128322FF30E10712831944203F
:109380008009EF30E2081283194440121B15F1B036
:10939000240B12832290261412BF49EF81ABF1B047
:1093A000240A128322FF540FFDEFC4540FFCEDC3B7
:1093B0009C400281B0F1B012C10C12D0A76F6002C4
:1093C00081B0F1B0240912832230E05D12C26A50EC
:1093D0000912831912D09E7405F0EC1490261BB567
:1093E000050512C1FD800A121E71E912C10CE924A3
:1093F00001128322FF9026141288C9ED6002818435
:10940000F1B0240912832230E37AF1B0240A1283E6
:1094100022F1AA12C0FF121AAD540F7067E924019D
:109420001283225418605D8053ED90261B70081241
:10943000C1FDF9E43A800E121E71E912C10CE92453
:10944000FFF9EA34FFFA121AADFF9026141288C908
:10945000EC146D702FF1B0240912832230E325F152
:10946000B0240A128322F1AA12C0FF121AAD540FBF
:109470007012E92401128322546060081283194497
:1094800004121B15902003E06008902016E0700283
:10949000A114F1B0240512832290261430E607129D
:1094A000831C4414800512831C4410121B15806415
:1094B000F1B0240A128322540FFD12C26A5055F1F2
:1094C000B0240912832230E023ED2402540FFDF171
:1094D000B0240A128322C4540FFFEDC39F5035F10C
:1094E000B012C10C12D0A76F702A801FEDC3940276
:1094F0004022F1B0128FD6ED24FEFFE434FFFEE9E6
:109500002FF9EA3EFA12D0A7B5070912831912D033
:109510009E7401F0F1B02404128322FF90121CE02B
:109520006F603012832A4A7002C1E712832A128FB9
:10953000BF12A83C12D0D712A7E86002C1E712837D
:109540002A24B6128322FFF1B024041283226F6012
:1095500002C1E712C26A4002C1E7F1B0240A1283D5
:1095600022FF540F1283294A7002C1E7E924BA127C
:109570008322FDF1B024082183226D6002C1E7F14E
:10958000B0240912832230E018EFC4540F24FE5493
:109590000F6E6002C1E712831912D09E7403F0C1EE
:1095A000E7EE64016002C1E712831912D09E7401D4
:1095B000F0C1E7F1B02408128322FF90121CE06F83
:1095C0006006EFF46002C1E71283194401121B1513
:1095D000F1B02404128322FF9026141288C9F1B03E
:1095E0002409F9E43AFAC003C002C00112B74712D5
:1095F0001EBA90261B12831C24F612BF3E1288CF7F
:10960000F1B0240512832220E602C1E71283194437
:1096100004C1D7F1B02408128322FF54E0FD901258
:109620001CE0D39D5002C1E7EF541F75F008A47CE5
:10963000002DFFEC35F0FEE0D39FEE12339F400289
:10964000C1E7F1B0240812832254E0FF90121CE01D
:10965000C39F14FFF1B02409F9E43AFAEF12CDE206
:10966000129F5EFEEF540712AD8C8002C333D8FC0C
:109670005E60741283194410121B15F1B024081295
:109680008322541FF1AD240912C101C003C002C0DE
:109690000112B747121EBAF1B02408128322541FD8
:1096A000FF90261B12831C24F6C39F12BF3EF9E4D1
:1096B0003AFAEF802212C28B6009902009E054BF71
:1096C0006F7024F1B02408128322FF90121CE0B5C1
:1096D00007151283194403121B15800B90261412D0
:1096E0001E711289BB9204F1B02405128322FF542B
:1096F0000F64016002E1A1EF90261B30E71412D045
:10970000DD128322F1AA12C0FF121AAD90261AF0C0
:109710008015121E71E9240912832290261AF0A3E3
:10972000121E7112BECEFAE924011283229026196C
:10973000F0128319FF300E6954E264807063902642
:109740001AE064017053902619E0640860533010E9
:1097500010F1B02409F9E43AFA12B74D12A7DC600F
:1097600030F1B012D0752404128322FFF1B012D070
:109770007524031283224FFFF1B012D07524051215
:1097800083224FFFF1B012D07524061283224F704E
:1097900008902619E06403600812831954EA121B2A
:1097A0001512831930E002D20422C4540FFF7E0048
:1097B00090261B121E71E92290276C121E917E00CA
:1097C0007F04122FF790276C129F9712AFEC74044E
:1097D000F012311E7F01227F0112CA32E49002B6DC
:1097E000124C27129F80E4FDF1B812CBEE7E007F71
:1097F00000C006C374079400FE7412940090267B88
:10980000F0A3CEF0124CACD00612311E1221FB1286
:10981000CB48124C2E1255CF79B602900312832AF0
:1098200024B7128322FF20E70201B6540F640160BF
:109830000201B612832A24B6128322FF90121CE082
:109840006F70732000709026E404F012832A24BB0A
:1098500012832230E34212832A24BC1283229026F0
:10986000E112D04124BD12C101121AAD540F70286B
:1098700012832A2FF9EE3AAFE924BE1283225460F4
:10988000601612832A24BC128322C4540F2404F1CC
:10989000527D6E7C0002B85AE4902008F012832AB0
:1098A00024BC128322C4540F75F03EA4FDACF07E9C
:1098B000197F8F0287CD12832A24B712832220E7D3
:1098C00016902104E0F46002D17812832A24B2F9C0
:1098D000E43AFEAF01D114F1387F019027C8EFF0D0
:1098E00012832A4AC36001D35037124CC3E4902636
:1098F000E4F012832AB1B5121C1245F0601A9027C9
:10990000C8E09026E16008B1B1D128E4FF8006B13B
:10991000B1D1287F01121F33124CAC9026E1121EE8
:1099200091229025FF12A8427B018B3F8A40F5418E
:10993000EDD394085002A18512831FFFEDC39F5001
:1099400002A185E4F546900413E0902002F0F1872F
:10995000D121E0B19DFF540F6401704CEF30E70F4F
:109960009025FFA3E0FF240AB1A112D02E8004F1BC
:10997000493540FA1255BE092607121E9190260756
:10998000124484FF601D64186019EF64076014EFCF
:10999000B40315902607F173F9E43AFAF17A12A7A5
:1099A000E870057FFE12A22B7B007A00793F1290AF
:1099B0002DB186902100F0E54644016062A202E4E8
:1099C00033F53EE4902605F0902605E0FFC39402AF
:1099D0005020EF12D0CAFF902100E0FEEFB5060A3A
:1099E000902605E024FF92028008902605E004F00E
:1099F00080D6902605E0B40206E53E24FF92029050
:109A00002002E0FDA202E43325E0FFE433FE74B05F
:109A10002FF58274213EF583EDF0A202B39202E5A8
:109A20004620E20241E47F01124C45902601F1906C
:109A3000700241E4B1A87F03128339B1BCB18C300C
:109A4000E40DB1A8E924B71283224410121B15B10A
:109A5000A8E91287F1E4121B1590260112BF559058
:109A60002601B1B1741975F07B121C3DB1A8E9242F
:109A7000BAF9E43AFAE547211B159026011287FD51
:109A8000121C12F1A6FDEF4DF19EB1BCB18C30E578
:109A90000FB1A8E924B71283224420121B15803687
:109AA000AB42AA43A944121AAD64017029E924010A
:109AB0001283226418701FE545B4040DE5442403A5
:109AC000F1651245198F1A800DAB42E5442402F16D
:109AD000651247A88F1AB1A8124CC79002B0E07067
:109AE00003122CC9200402816BE546544264407085
:109AF0001D9026E4E070028186E4F15212832A244C
:109B0000BC12832254F0FD7C001287CD8186E5468D
:109B100020E10261DDE4F53E12832A24B71283229C
:109B2000FF540F6401600261AEEF30E77712832AC1
:109B300024D8128322FFD3940A400A12832A24BC19
:109B4000128322800490210EE0902606F0902606D3
:109B5000E0FE540FFD902605F0BD0F028037EFD3D5
:109B6000940A401312832A128FC6902605E07C00C7
:109B700029F15EF53E8010092605E0240FF582E408
:109B80003421F583E0F53EEE54F0C4540FFF9026E7
:109B900005E0B5070A12832A24BA128322F53E1281
:109BA000C4F5800A12832A24BA128322F53E128356
:109BB0002A4A70028186B186653E6008902016E0D0
:109BC00070028186B1BCB18C30E70CE5412409B14B
:109BD0008C540624FF9200111DC2008186E5465474
:109BE00022FFBF20129026E4E070028186D121E09E
:109BF000FFD114F11E8186E54630E4028186902073
:109C000016E030E2028186AB3FE5412408B18CF4D6
:109C100060139025FFB198540FFDBD0203D380015E
:109C2000C34002D114E54630E30BD121E0AA06F986
:109C30007B0112A36F20274EB1C3902604EFF07A68
:109C400020790F7D06128000902604E0FFB186FD8A
:109C50009025D6E545F07B017A20790FA3121E915D
:109C6000AB42AA43A94412B009801BF18AEA494BCE
:109C700060149026E0E060E090200EE06008124260
:109C800032E490200EF0E54620E409902016E02012
:109C9000E202A185902003E06002A183902002E00F
:109CA000F53ED2057B017A207904128F3612D0EB73
:109CB000AB3FE541240AB18CFF540FFEE541240976
:109CC000B18CFD30E01A1EEEB4FF0AE5412405B167
:109CD0008C44408006B1BCB18C54BF121B15803837
:109CE000EFC4540FFF146E702EED30E32AEFFD7CAD
:109CF00000AB3FE541240BF9E43540F15B540F70B4
:109D000016E924011283225460FF600BBF20054333
:109D10003E208003433E400EAB3FE541240AB18C18
:109D200054F0FFEE540F4F121B15AB3FE5412407D3
:109D3000B18CFF740AD39F4005740A121B15121AC6
:109D4000AD24F6FFF1493540128F35D11A128F42FA
:109D5000C203B186FDE5412408B18CFBC003D11AD2
:109D600012A369AB3FE5412407B18C24F6902594FA
:109D7000F0A37481F0A37491F0A37499F0D003AFB1
:109D80003EE140C20522AB3FE5412404F9E4354001
:109D9000FA021AADF090271AE0FEA3E0FF7B01243F
:109DA00005F9E43EFA021AAD902601021E719027D1
:109DB00087121E71E924DCF9E43AFA22AB3FE5414F
:109DC00024052212CBDDEF60047F0180027F00B109
:109DD000BCB18CFD30E504EF4402FFE54630E704FA
:109DE000EF4480FFED540FFDBD0506EF4410FF80EA
:109DF00022BD0111AB3FE5412408B18CB4FF14EF43
:109E00004404FF800EB1BCB18C540FFDBD0204EFC1
:109E10004408FF2212AAA702A8AE7B017A21790D7D
:109E2000229025FFE0FEA322121C12F58285F0830A
:109E300022902787121E91902787F1731283223078
:109E4000E019D172E924B7128322540FFFBF050332
:109E5000D38001C34005D17202874EB1AE121C12ED
:109E600045F06009B1AED128E4FF121F33D1720270
:109E70004CC3902787021E17902106E0FF7403A8A9
:109E800007088002C333D8FCFE902015E0F114E0EF
:109E90005EFEA807088002C313D8FC902772F0E486
:109EA000A3F0A304F07E03902773E0FDC394045055
:109EB00062902015E0FCF114E05EFBA8050880022A
:109EC000C313D8FCFDC394004016902772E0FBED4D
:109ED0009B500D902774E0FD74172CF116E02DF0C7
:109EE000902015E0F114C083C082E0FD7403A80740
:109EF000088002C333D8FCF45DD082D083F0902771
:109F000073E004F0EE25E025E0FEA3E025E025E087
:109F1000F08094222417F582E43420F58322128302
:109F20002A240212832230E209902104E0F4600224
:109F3000D178F1387F0101DBE49026E0F00242287D
:109F400012A2DB902003EFF022AB3FE5412409F998
:109F5000E422902008F07E197F8F22FAE92DF9EC97
:109F60003AFA021AADF9E43543FA121AADFF22F0BB
:109F70009025D3121E71E94202229026AB121E9147
:109F80007B017A0279B622C21D229026E1021E715F
:109F9000121E91EA494B227E007F00021E71FFE5EE
:109FA000F08FF0021C3D54F8FF902002E0220227BF
:109FB0003C122FF7E433FF229026CDE09026C1F02B
:109FC00002275C90269EE0FDA3E090267BCDF0A3C7
:109FD000EDF012311E500990269FE02401FF80020F
:109FE0007F012290260FE0FDA3E090269ECDF0A3F6
:109FF000EDF0F1C3902613EFF090261112A00D6042
:10A000000312448A902613E0FF22902383E0FEA3EC
:10A01000E0FF4E229027C112277A11F01168902795
:10A02000C1E06405701F740411AF9023D27419F05D
:10A03000A374DFF074013104110A602B8F828E83C8
:10A040007F05021F339027C1E0700D9023D6741353
:10A05000F09023D47403F022110A60098F828E835A
:10A060007F04121F3311AA229026B1ECF0A3EDF069
:10A070009026AE121E9112A1ADFFF46003023FAD17
:10A080009026B1E0FEA3E0FF123FCE12448E902650
:10A09000AE121E71EF121B159026AE124484B4FF4F
:10A0A0000811AA110A6002510E2212C88D74019083
:10A0B00023D4F0E49023D6F0229027C012277A9080
:10A0C00027C0E0700411F0809F11AA110A600251AC
:10A0D0000E22EF701A9023D4E0B4040411F08088AB
:10A0E00011AA110A60098F828E83E4FF121F3322A6
:10A0F0007B017A2379D57C197DD59026B374FEF047
:10A10000A304F022902379F0E4FF31B0FF640460EF
:10A110006AEFB403028064902379E0B4010CC20EAC
:10A1200090121CE07004902379F0902379E0701D68
:10A13000FF12CA78C20EE49023B0F020100D9012E6
:10A140001DE0543070057F0112CD82C2109023D2E1
:10A15000E0FAA3E0FB4A6019902379B14EFD8B82AF
:10A160008A83121F33902379E070069023D2F0A3E4
:10A17000F0902379E0B401707403F07F0431E7229A
:10A18000AB05AA04902379E07021EF24FF920EEF33
:10A19000B40103D38001C39210300E139023D21266
:10A1A000422020100A753001C21322E4FF310A2236
:10A1B00031B7902379E0229023DFE0FFF4600312AF
:10A1C000442A9023DF74FFF022902378E0FF14F0FC
:10A1D000EF701331B0B403028007902379E0B40428
:10A1E00005E4F0FF310A229027C3EFF031B7902742
:10A1F000C3E06004902378F07E1A7F077BFF7D2FF9
:10A2000012448E9023DFEFF0BFFF0231C9228F820C
:10A210008E837F01021F339023D6E004F0D3941481
:10A220004008110A6002510E11AA229027ABEFF0EC
:10A2300090121CE06F6051E49027ACF09027ACE0E6
:10A24000FFC39402502BEF518D1244054E60115103
:10A2500089124405F58251105189F583E4F0A3F089
:10A260009027ACE012CD6BE4F09027ACE004F080D6
:10A27000CBC2159027ABE04BFE0E7FFE12CCFF1237
:10A280008FCDF876070876D0229027ACE075F04B9A
:10A29000A424C5F582E4342122902753F141F07BB8
:10A2A000017A2379E312C915902754E0FF30E502C3
:10A2B000D206EF54DF902754F0301111C211715EB5
:10A2C0007146F14C902753E0FB7F02800E9027539C
:10A2D000715A7146F1AB902753E0FB90258E1239ED
:10A2E000C77F02124C45902598129F90605390258D
:10A2F0008EE0FFA3E0FD902591F12F902594E09052
:10A300002556F0902595E0902557F0902596E0FB96
:10A31000A3E0902558CBF0A3EBF0902598121E7186
:10A3200090255A121E91902590E0FB128D5F90258A
:10A330009BEFF060037F0122902598121E71124C52
:10A34000C3F1237F002290240DE0902594F0902704
:10A3500054E0902595F090275522E0FFB1559012DA
:10A360001CE0FD7B017A2379E3902591021E9190F8
:10A370002747121E91902030E06002811E911F2419
:10A38000091283224401121B154402121B15911F4E
:10A39000240A128322FF540FFE90274AF0EF54F054
:10A3A000121B1554F0FFEE14540F4F121B15121A06
:10A3B000ADC4540FFF90274712831CFEC39FFFC3F9
:10A3C000EE9F240290274AF0D394A2400374A2F097
:10A3D00090274AE0FF911F2409128F32129E1A1211
:10A3E0008F4290210EE054F7F0C203902002B14E4C
:10A3F000FD911F2404128322FBC003129E1A71696F
:10A4000090274AE090259412C07DD003129F40907F
:10A4100002B0E07009902003E06003122CC9229082
:10A420002747121E71E9229027A3EFF012B692126D
:10A43000B7A733333354F89027A4F0200F0281DFFD
:10A440009027A4E0FF9027A3E0FEC39F5051EE1396
:10A450001313541FFF12A84BA312A895E0FD7C0014
:10A46000EE540712BF878005C333CE33CED8F9FF31
:10A47000EE5CFEEF5D4E60F19027A3E09023D7F0F5
:10A4800012457CAD079023D7E004FF7A197BEE914B
:10A49000E2EF704D02C8E29027A3E004F080A1C271
:10A4A00018C20F9023DA7401F090237AF0A3740796
:10A4B000F0E4A3F09023797403F09023D8B14EFD1B
:10A4C0007B017A23797A71699025947403F0902343
:10A4D0007F12D09090237EB1D870067F02210AC2ED
:10A4E000182290274FF141F090237A7401F0A37461
:10A4F00018F0902750E0FF12479190237CEFF090E6
:10A500002750E090237DF07552019023DAE0FFB4EC
:10A510000203755202EFB403037552039023B0E0B7
:10A52000FF600C7F40B402027F20EF4402F552909E
:10A53000121CE0FD7B017A23797A71697404F13889
:10A54000902751F14C90274FE0FBAF5241DBE0FFE9
:10A5500090121CE022E4FEEE12D0CAB5070FEE25E1
:10A56000E024B0F582E43421F583E0FF220EEEB45E
:10A5700002E57F012290275AEFF0A37407F09023A1
:10A58000E1E06004F12860037F0022F1877415F098
:10A5900012CBD6128F360B7A2379E57F05128F42C4
:10A5A0009027A5E0600C9023EA74FFF09027A6E0C6
:10A5B00004F09023E1715A9027A6E0902594F0A32F
:10A5C0007405F0A37419F0A374DAF09023E1B1D804
:10A5D000700302D0B07F0122E0FB51DBEF22902715
:10A5E000C4EFF0F12860037F0022F1877416F09029
:10A5F000121CE09023E5F09027C4715A7403F138DF
:10A60000A37419F0A374E4F09027C4B1D8700302C6
:10A61000D0B07F0122902657121E91AC0790265B86
:10A62000E05437F030E502D20690265BE04420F09B
:10A63000C201AF04F11BAE04AB06C0039026571253
:10A640001E71716990265AE0902594F090265BE087
:10A65000902595F090265CF1ABD00341DB9025600E
:10A66000121E91902563EDF0A3121E71E9240112D0
:10A67000832230E502D206F702124C4590256C1277
:10A680009F907002E11090256C12B68B12832244C9
:10A6900008121B15902567E0FEA3E0FFF115E924E1
:10A6A000E0F9E43AFA12BA09902569121E71C00362
:10A6B000C002C001F115E924E2F9E43AFA121EBA27
:10A6C000902564124484FFF11B902564124484FB9E
:10A6D000C003902560F12F902563E0902556F090FF
:10A6E0002564121E71E92401128322902557F0E49B
:10A6F000A3F0A3F0F11590255A121E91D003128DEC
:10A700005F90256FEFF060037F0122F115124CC3BB
:10A71000F1237F002290256C021E71B15590121C0E
:10A72000E0FD22C206D203229023D4E0640122126B
:10A730001E71902553021E91902594F0A37411F080
:10A7400022EFF0A3EDF0A3EAF0A3EB22E0FFA3E0F9
:10A75000902596CFF0A3EFF0229027A9ECF0A3ED7F
:10A76000F19604F0D20690121CE0FDAB07C0037115
:10A77000639025947402F03A7405F09027A9F14C87
:10A78000D003F19F24FF229023D47402F0AF0590F0
:10A790002383ECF0A3EFF09023E37401F0A322E411
:10A7A000FF51DBEF2212D086F081E2E0FBA3E090C4
:10A7B0002596CBF0A3EBF0229026A8121E91AE07AF
:10A7C0001FEE60159026ABE4122749FE9026A8E400
:10A7D0001227496E60E87F01227F00229026AB128B
:10A7E0001E917B017A2079047F04F1B8EF22902733
:10A7F000AD12A8427B01C002C0017A0279B612A84C
:10A800003CD001D00212A7E87002D3229027ADE01D
:10A81000FEA3E0FFF5828E83A3E0FD8F828E83E0AE
:10A820004DFF9027ADE0FCA3E0FD1152E04FFF8DFE
:10A83000828C83A3A3A3E04F24FFB3229026AB0214
:10A840001E91EEF0A3EFF0AA06F9229023DBE0FCC4
:10A85000A3E0F5828C83A3A3229023D7E09027C2A4
:10A86000F0EF6028E0FF131313541FFE114BA3E514
:10A87000822E1198C083C028E0FEEF5407B18C806F
:10A8800002C333D8FCF45ED082D083F09027C2E0BC
:10A8900004FF02A427E5822FF582E43583F58322A5
:10A8A000F9E43AAD01902785F0A3EDF0916590278A
:10A8B00057EFF0C3940240024198902757E02419C3
:10A8C000B140E0FF90275AF09023E1E0FEEFB5069B
:10A8D00005E4F54C800690275AE0F54CE54C75F000
:10A8E00011A42407F9740035F090275A122FF2E5CD
:10A8F0004C12272C8F52E5525403FF602F9027579C
:10A90000E0FE519DE0548FF0741E2E519FE04420D4
:10A91000F0902757E0FE915BE0549FF074172E9162
:10A920005DE0FEEFC43354E0FFEE4FF0E4902759B2
:10A93000F0E4902758F0E54CB17CFA902759B159D2
:10A94000FA902758B19512273C8F52902757E0FF75
:10A95000519DE0540FFE902758E0FDC39E500EEF2E
:10A96000B12FE5822D1198E0FD7C00800F902758D3
:10A97000E07005FC7DFE80407C007D00AF05EF654A
:10A980005260028023EF64FE70024198902758E0E5
:10A99000FD6009EF7006EE6D70024198902758E057
:10A9A00004F0E0C39404408E902758E064047002E1
:10A9B0004198902759E004F0E0C3940450022131FB
:10A9C000E54CB17CAF01F54A8F4B5199E0540FF53E
:10A9D00052E4902758F0902758E0FFC39404501990
:10A9E000AD4C12CFE9ACF0E54CB17C12B6E9EF60AA
:10A9F00008902758E004F080DD902758E0C39404C5
:10AA000040037403F0902758E0FFAD4CB1A09027AD
:10AA100058EFF05199E0540FF552E4902759F0E5C2
:10AA2000527009B148FEAF017DFE801C902759E0AD
:10AA3000C39552501EB148B193E0FD902757E0B145
:10AA40002FE5822D1198E0FD122FF7902759E00491
:10AA5000F080D9902759E0C394045009B148B193CC
:10AA6000E4FD122FF7E54C12C1F31227358F525136
:10AA700099E054F0C39402050DB1888002C333D825
:10AA8000FCF45252800AB1888002C333D8FC42528F
:10AA9000E54C12C1F312C20422902757E0241EF5A0
:10AAA00082E43412F5832290271AEEF0A3EFF0200F
:10AAB0001D0F902002E0B4010B9153129D9D20E7E1
:10AAC000037FFF2291537B012404129DA1FF90126A
:10AAD0001CE06F6002800A91537B012408129DA143
:10AAE000FFAD0712CB2390271EEFF0F4704CF1AEB0
:10AAF0005033E004F0E490271EF090271EE0FFC3DF
:10AB00009402500DB13DE0600890271EE004F080F3
:10AB1000E990271EE0B402037401F090271EE024A0
:10AB2000FF921C8015201E0CB21CA21CE43390273F
:10AB30001EF0800690271E7401F090271EE0241955
:10AB4000B140ED129D9420E70261EDEF2409129DC2
:10AB5000A130E32190271AA3E0240A129DA112D06C
:10AB60002EFAE924011283225418FF90271EE09147
:10AB70005BEFF080089027E1E0915BE4F091537B7C
:10AB800001240A129DA1C4540FFF90271E519CEF6F
:10AB9000F090271AE0FCA3E0240BF9E43CAD01A3FC
:10ABA000F0A3EDF090271AA3E02409F9E43CFA128F
:10ABB0001AAD20E018AE071FEE604812CFDFB16774
:10ABC000FE90271EE0B12F1195EEF080E8E4FEAD77
:10ABD000071FED602E12CFDFB167FDAC060E902788
:10ABE0001EE0B12FE5822C1198EDF080E290271E37
:10ABF000E0FF519DE4F074172F915DE4F0EFB12F69
:10AC000074FEF090271E519CC083C082E0FF90200C
:10AC100002E012BF37D082D083129D9430E709EF53
:10AC20002409129DA120E4089153129D9D30E40C4B
:10AC300012CDD28002C333D8FC4F800B12CDD2800C
:10AC400002C333D8FCF45F90121BF0D21D90271E74
:10AC5000E0FF2290271AE0FEA3E0222417F582E409
:10AC60003412F58322AD0779FF301D02A12B12CBE0
:10AC700023A907EFF470271FAE501AE004F0E4F99F
:10AC8000741929B140E0600509E9B402F3E9B4029E
:10AC90000D79018009201E04E4F9800279017419FC
:10ACA00029B140EDF0741729915DE4F0902785E01B
:10ACB000FCA3E0F5828C83E0540FFE741E29519FA3
:10ACC000EEF0741E29519FC083C082E0FD902002E7
:10ACD000E0C454F0FCED4CD082D083F0EE602DE463
:10ACE000FDAC061EEC602A902785E475F00130313A
:10ACF0000DB164FCAB050DB12EE5822B8008B1646B
:10AD0000FCB12EE5822E1198ECF080D5B12E74FEA8
:10AD1000F090121BE0FEAF017401A807088002C387
:10AD200033D8FCF45E90121BF0D21DAF0122E9254E
:10AD3000E025E02423F582E43412F5832274192FF0
:10AD4000F582E43412F58322E54C75F011A4240851
:10AD5000F9740035F0FA902758E075F004A429F949
:10AD6000EA35F022121BE685F082F583E022B1A0DD
:10AD7000EF75F004A4FDAC0F902015E075F011A460
:10AD80002408F9740035F022902758E0FF7401A8D8
:10AD9000070822FAA3E07E0029F9EE3AFEAF01226D
:10ADA000E4FE7C03EEC39404502A74172D129F1600
:10ADB000E05CFBEE25E0FAEBA802088002C313D8A2
:10ADC000FCB50707902106EEF0FF220EEC25E025EA
:10ADD000E0FC80D07F00229027BCEFF09027BCE001
:10ADE000FFC394045055902015E0FD7880F6B16EB5
:10ADF00012B6E9EF603D12CFF3FDB16EFAE92DF91D
:10AE0000EA3C12D01E12275C9027BC12D01464FEBC
:10AE10006029E4FF74822FF8E6700E9027BCE06092
:10AE20001AEF701774FFF080127881060FEFB404E8
:10AE3000E380089027BC7404F080A19027BCE0C395
:10AE40009404400574FFF0804490201512C1F21262
:10AE50002735A90712CFF312CFFD8002C313D8FC08
:10AE60005403600D24FE600F1470127886761880EB
:10AE70001078867620800A87867610800478867619
:10AE80000890201512272BEF600312D00C9027BCDE
:10AE9000E0FF229027BD12CB5A12C90D50557E00FB
:10AEA0007F0712273C7880EFF660409027BDE0FFD7
:10AEB000E4FDB1A0EF75F004B17F12D01E12275C43
:10AEC0009027BD12D01464FE6029E4FF74822FF82D
:10AED000E6700E9027BDE0601AEF701774FFF080E7
:10AEE000127881060FEFB404E380089027BD74FF49
:10AEF000F080A612C90D400574FFF080517B027AE4
:10AF00000F79807E0F7F8012273CA9079027BDE034
:10AF1000FFE412CFFD8002C313D8FC7E0060047FE3
:10AF20000180027F00EF7803C333CE33CED8F9FF20
:10AF30007886F6BF10117B027A0F79817E0F7F81B0
:10AF400012273CEF12D00C7886E67002762090270C
:10AF5000BDE0FF229027BE12CB5A90201574FFF05F
:10AF6000902104F09027BEE0B5070AE4902015F088
:10AF7000FFD19380239027EBE0FDE4FF12CFE9ACF3
:10AF8000F09027BEB17B12B6E9EF60119027BEE0CA
:10AF9000902015F0E4FFB1D7902104EFF090201538
:10AFA000E0C394FF50028001C322E4FF01599012D4
:10AFB00016E0C3940222E4902797F0A3F020270222
:10AFC000C322902797E0FEA3E0FFC3EE9440501405
:10AFD000F1E67420F012311E902797E475F02012EC
:10AFE0001BE680DED3227B007A00790090267BE48A
:10AFF000F0A3227E117F52F1E67405F012311E1289
:10B00000CBD67D05E4FF0280049025D1EFF0A3EDBF
:10B01000F0A3121E919025D6E0FF7401C39F400259
:10B02000C1809025D7121E719025D7121E919025B0
:10B03000D3124484FEC39420401EEED394FF5018D4
:10B04000EF949F50139025D1E0FFA3E0FD9025D60B
:10B05000E0902584F0021A989025D312448464016C
:10B060006002C180E92401128322121F09B59101F7
:10B07000B0CC02B0EA03B3AE04B4E405B09508B3B3
:10B08000B90BB1B90CB31F14B16216B1A517B676DE
:10B09000220000B680300F02C180200E02C18090D5
:10B0A00025D6E0C394035002C180129F7012832200
:10B0B00020E002C180D2119025D2E0FF9025D1E09E
:10B0C0007D1030E1027D12E4FBFA801B9025D1E077
:10B0D00030E10AA3E0FFE4FBFA7D07800A9025D265
:10B0E000E0FFE4FBFA7D0502A299300F02C1802047
:10B0F0000E02C1809025D6E0C394074003D380019F
:10B10000C34002C1809023797401129F6F12832281
:10B1100090121CF0D182128F2F129F807F04128F09
:10B1200042129F8090121CE0FD1297B890121CE012
:10B13000700612CBEE12C51790121CE0701C12AFF5
:10B14000F37E007F07124CAC90267B7411F0A37441
:10B150004BF012311EE49023E1F0E4FF12A10A0249
:10B16000CB0190121DE020E002C1809023E1E0FFBE
:10B1700070057552018002F852129F70128322905E
:10B1800023D912A7967416F09023D9E09023E5F006
:10B1900012A35E12C8D7A37419F0A374E9F0AB52DE
:10B1A0007F0102A2DB9023D4E064036002C180121D
:10B1B0009F70128322FF02A014C2D57552FFD1885E
:10B1C000128322FFC454079025DBF0700C129F708D
:10B1D0001283229023E0F0D2D59023E0E070024168
:10B1E000D7E4F54C744D254CF8E6FF9023E0E06F72
:10B1F0006012EF7008E552B4FF03854C52054CE530
:10B200004CB405E0E54CC394054022E55294FF5050
:10B210001C9023E0E0FD744D2552F8A6057E0074D5
:10B22000522552F9EE3411FEAF01122FF79023E0B0
:10B23000E0FFF1AF9025DBE0C394044002611230DF
:10B24000D50312B8AF30D50CD1ADAF019023E0E0FB
:10B25000FD122FF7D1881283225407F552E490256E
:10B26000DCF030D519E5527015AE4AAF4BFCD1A0D9
:10B27000FA9025DB12AD59EFAF017DFE80279025B6
:10B28000DCE0C395525029D19AFA9025DB12AD59D2
:10B29000FAA3E0FD29F9EC3AFEAF019025D312871D
:10B2A000FD129F5CFD122FF79025DCE004F080CEAC
:10B2B0009025DCE0C394045011D19AFA9025DB125A
:10B2C000AD5912AD93E4FD122FF7D1829023E0E047
:10B2D000FD12D07D02C11B30D538E4F54AF54BD1C3
:10B2E000ADAF0112273CEF6015D1ADF156E4F54C3E
:10B2F000D19AFAE54C12AD5AF155F18E40F2054B58
:10B30000E54B7002054AC394E8E54A940040D01228
:10B31000AFF312A7287002C18012A0F002A068D17A
:10B3200088128322FFC45407FE9025DBF0EF5407F8
:10B33000F552EE70177FE812B8AF129F7012832299
:10B340009023E1F0FD7E007F07122FF79025DBE0D0
:10B35000FFC39404505EE5526019EF75F00412AD1E
:10B360007FFEAF019025D31287FD12AFECE552F0BE
:10B3700012311EE552700E0925DBE070087E007F59
:10B38000087DFE801CE552C3940450189025DBE034
:10B3900075F00412AD7FFA7E00E9255212AD99E4F2
:10B3A000FD122FF79023E1E0600AD18212D07DE4F4
:10B3B000FD12C11B7F0302A1E712A7287002C18002
:10B3C00012A0AAE4902379F012A1B7F15D90238333
:10B3D000E0FCA3E0FD4C7002C180129F701283223A
:10B3E00024FEFF8D828C83021F33300F02C18090B8
:10B3F00025D6E0FFD394224002C180EF940350028F
:10B40000C180129F70128322D3941D4002C180908C
:10B410002002E09023D8F0740212A104D20F9023EE
:10B42000D4E0B4040312C88D12CB0112D086129F4F
:10B430006F128322FF541F2403FDE433FC9025D6B2
:10B44000E0D312339D400E7E00D18812C101121A42
:10B45000AD9023B0F09023B0E070067E247F0E8084
:10B46000047E237FB19023DB12A8427B01C003C07E
:10B4700002C001D182128F63D001D002D0037F219C
:10B48000128F42129F70128322541F2404FFE43350
:10B49000FE9025D6E0D39FEE12339F400FD182E974
:10B4A0002FF9EA3EFA121AAD9023DAF09025D2E095
:10B4B00090237EF0A3F19E30E10790237FE04402C9
:10B4C000F0D218D192FF2403FDE43EFAA9057B01D6
:10B4D0001238DCE0FD12CE11EF2407902378F0E45F
:10B4E000FF02A4279023797404F012A1B7E49023FB
:10B4F000B0F09025D6E0D39402400A129F701283D8
:10B50000229023B0F09023B0E0FB70067C247D0EE7
:10B5100080047C237DB19023DBECF0A3EDF0F58279
:10B520008C837401F0A37406F09025DAF19E30E16B
:10B53000079025DAE04402F0D192F1A670051238A6
:10B54000DC04F0D192F1A61238DCA3258212A8986F
:10B55000EBF090121CE0FDD192FFAA06F97B0112DC
:10B56000A3691238DCE02404FF9023B0E07E007071
:10B57000027E01C3EF9E905294F09025DA12D09093
:10B580009025D2E0FB12A79F6002C1807F0202A13A
:10B590000A9025D6E0FFC39406E494005002C180CF
:10B5A0008F4C7A23798D7D23128000D188128322DB
:10B5B000FF20E25D4404121B15D182128F367B01FD
:10B5C0007A2379857F06128F4290238AE0A3F0D1F7
:10B5D000F5E490238CF0054C054CF196E434FFFE25
:10B5E000D3EF9400EE94004075D3EF9423EE9400D3
:10B5F00040037429F0F1969025D312BF42128F3286
:10B600007B017A23798D128F429025D6E0F54C800C
:10B610004D9025D6E0D3942B4005742BF0F54C903B
:10B6200025D6E0D181128F367B017A237985128F5E
:10B6300042902388E020E126D1F59025D6E0B42B76
:10B640000414F08002054C9025D6E024FBD181E95A
:10B650002405128F327B017A23798B128F42902539
:10B66000D2E0FD7B017A23798AE54C24FB9026F118
:10B67000F07F84021A9D12F970128322FF12CD828C
:10B6800022FF9025D3021E719025D3121E71E9244A
:10B6900003229023DBE0FEA3E022AE4AAF4B7C0006
:10B6A0007D11121B4974192FF974003E22AE4AAF66
:10B6B0004B7C007D11121B4974182FF974003EFE5B
:10B6C00022EF7002C322EFF1AFFED19CD1EFEF6009
:10B6D00016E4F54CD19AFAE54C12AD5AD1EFBFFE03
:10B6E00002D322F18E40EDC322FAE92DF9EA3CFEA5
:10B6F000AF0102273C7B017A237987902781121EB4
:10B7000091902781121E71E92401128322FF30E1FA
:10B710001890278112448430E706F14D7402801A94
:10B72000902781F14A74018011EF90278130E30660
:10B73000F14A74048004F14A7403121B15902781A6
:10B74000D18B128322FF22902614121E71E924034A
:10B75000F9E43AFA22FEAF01E4FD022FF712CBD250
:10B760009026C17405F012275CE4F54C744D254C0D
:10B77000F8E6D394E8400D4EF6FE7452254CF9EEEF
:10B780003411F155054CE54CC3940540DF22054CBE
:10B79000E54CC39404229025D6E024FAFF227401DC
:10B7A000F09025D1E022FFF5828E83A3A3E022242E
:10B7B000FFF54BE434FFF54A222290276F121E91C9
:10B7C0007F0112277EF1EE121C1245F0601F9027B8
:10B7D0006F121E71C003C002C001F1EE128FF9F5A5
:10B7E0008285F083D001D002D003121F332290272C
:10B7F0006F121E71E924DAF9E43AFA22902799EEE1
:10B80000F0A3EFF012832A128801121C125407FFD2
:10B8100064026005EF64037016115125E0FBEC3300
:10B82000FAEDAE047803C333CE33CED8F9801C11C1
:10B8300051AE047803C333CE33CED8F9FBAA06ED5C
:10B84000AE047805C333CE33CED8F92BFFEE3AFEE3
:10B8500022902799E0FCA3E0FD229026E07401F0FD
:10B86000C006C007EDAE047803C333CE33CED8F99B
:10B87000FBAA06AE04ED7850C333CE33CED8F92BF5
:10B88000FDEE3AFCD007D0060241937B017A217984
:10B890000C024441E49027BBF0F09027BBE0FFC3CB
:10B8A00094E9500A11AF9027BBE004F080EC2274B9
:10B8B000172F129F1674E4F022123FFBEFC4540FAF
:10B8C0006FFEEFC41354076EFEEFC413131354013D
:10B8D0006E5403FF22128800EE8FF0021C3D90266A
:10B8E000DB121E919026DAEFF09026DE7402F0EF64
:10B8F000700221ED901216E0700221ED9026DEE03C
:10B90000FF2418F190FE9026DAE06E600221E33108
:10B91000F7FE540F9026DFF09026DB1287FD121CF5
:10B920001254F8FDEEC4540FFFE5F0FEED4F510840
:10B9300031F1128FF7EF549FFF9026DEE02416F5C9
:10B9400082E43412F583E05460FDEF4D31F011D5FF
:10B9500031F1E9128FC6C003C002C0019026DEE0BB
:10B9600075F004A4241FF9741235F0FA7B01128FCC
:10B97000369026DFE0FFD010D002D003128F429025
:10B9800026DFE0C454F031F0E924BC1288CF9026C1
:10B99000DEE014F1878005C333CE33CED8F9FF90B3
:10B9A000121BE0FDEF5D60389026DB12B68B128330
:10B9B000224404121B159026DEE0FF241D31FA54A8
:10B9C0008FF031F74430F090121BE0FF9026DEE05C
:10B9D0001412CDDB8002C333D8FCF45F90121BF04D
:10B9E0007F01229026DEE014F0600201FC7F00223D
:10B9F000FF9026DB021E71741D2FF582E43412F5D0
:10BA000083E022EF54F84402FFEE8FF0021C3D90D9
:10BA100025AAEFF0A3EDF0A3121E919025B0E0FF50
:10BA20009025B3129F731288CFEF7E0030E1047F20
:10BA30000880027F009025B31287FD51099025AF41
:10BA4000E0FF74A9C39F500374A9F09025AFE09064
:10BA500025B3F149C003C002C0019025AC121E718C
:10BA6000128F36D001D002D003128F429025AFE062
:10BA7000FF716BE924B11288CF9025B1E0FEA3E0FD
:10BA8000FFA3129DB151099025B3F1559025AAE06D
:10BA90009025B6F09025ABE0540FFD640260317143
:10BAA0006BE924BA128322F53EB4FF0B9025B6E071
:10BAB00054F84401F080199025B6E0FF5407701047
:10BAC000902100E0B53E09EF129FA64F9025B6F0F9
:10BAD0009025B31287FD121C1254EF129F9E300363
:10BAE00031ED6404600A9025ABE0540F6406700FDA
:10BAF0007171BF0203D38001C39223D224800D71E0
:10BB000071BF0203D38001C39223C2247182EE4F1E
:10BB100080089025ABE0F176F1379025ABF0D203A9
:10BB20009025ABE0FF716BE924B71288CF540F1258
:10BB30001B15122F1F9025B6E0FF9025B31287FD2D
:10BB4000E48FF0121C3D9025ABE0FF716B1283393E
:10BB50009025B31287FD121C12FF9025B3F142F914
:10BB6000E43AFA129F9F716B024CC79025B3021EF4
:10BB7000719025ABE0FE9052B6E05407FF2292236D
:10BB8000C22420232A302413E54954F0FFBFF003D8
:10BB900053490F74102549F549803CE549540FFF7E
:10BBA000BF0F035349F00549E549540FC4802830BD
:10BBB0002413E54854F0FFBFF00353480F741025D9
:10BBC00048F5488012E548540FFFBF0F035348F073
:10BBD0000548E548540FC454F0FF229025B9121EC1
:10BBE000919025C07406F09025BCE0FE7411D39EA0
:10BBF000400281CB74409E500281CB7F02124C45A3
:10BC00009025C1129F90700281CB9025C0E0300337
:10BC10000CFED223D2247182EE4FF08011FF9025CA
:10BC2000B9F142128322540FF1379025C0F09025CC
:10BC3000BDE0FF9025C1129F731288CF9025C112DD
:10BC400087FDE475F002121C3D9025C1128FBBC028
:10BC500003C002C0019025B9121E71128F36D001A7
:10BC6000D002D0037F11128F429025BCE024EFFF59
:10BC70009025C1121E71E942B11288CF9025C1F101
:10BC80004AC003C002C0019025B9121E71E92411F7
:10BC9000128F32D001D002D003128F429025C1F111
:10BCA000559025BEE0FEA3E0FF9025C1129DB15145
:10BCB00009D2039025C0E0FFA3121E7112833990B0
:10BCC00025C1121E71124CC77F0122D2037F0022B0
:10BCD000E5336002A178B17AE9240412832290222C
:10BCE0005230E615123343E475F064121C3DB17A0C
:10BCF0007406121B15C2038030F1671283224420A0
:10BD0000B179E924141288CFB17AE9F17E121B15BA
:10BD1000B17AE9F1A1128004B17A7405121B159071
:10BD20002252123343F16ED203902252129F7312A9
:10BD30008322B179E92403128322FDB17A128FD5CF
:10BD4000C003C002C001B17AE92406128322902503
:10BD5000BCF0B17AE924041283229025BDF0A374CB
:10BD60001AF0A3742AF0D001D002D00371DBEF7077
:10BD700007B17A7407121B5122FF902252021E71E2
:10BD80007F337D3412CC3DE53314700312CC7EE456
:10BD9000F532E53275F04BA424BCF9742135F0FA84
:10BDA0007B01902252121E91121AAD24FE601524BE
:10BDB000FE60151460161460171460182406704B8A
:10BDC000D1668047D1D5804391D0803FD124803B3C
:10BDD000D1EB8037B17AD1CEFA121C1245F0602334
:10BDE000E5336404600AB17AE92401128322F53450
:10BDF000B17AD1CEFA129E28AF34121F33B17AE94C
:10BE000012D0BEB17AE4121B15C2150532E532C359
:10BE100094025002A192E5316009FD7F0112CC0429
:10BE2000E4F53122E53324FD602914601624037003
:10BE300034F1065030C214B17A1255BE7401121B8F
:10BE400015801BB17AE9240412832220E002800EBF
:10BE5000D21422B17AE92403128322B53407B17ACD
:10BE60007407121B1522B17AE4121B15B17AE9246A
:10BE700005128322146003407053B17AE92417122B
:10BE80008322540F9027C6F09022526030121E7108
:10BE9000E92416128322FF124006EFFD9027C6E028
:10BEA00014F075F064A42419FFE435F0CF2DCF34DD
:10BEB00000FE902252123343EE8FF080061233437D
:10BEC000E4F5F0121C3DB17A7402121B1522E9242C
:10BED00009F9E43A22E533147010F106500C2015EC
:10BEE00009D215B17A7404121B1522E53324FD60C2
:10BEF0000D14600A2403700DF10650098000B17A18
:10BF00007407121B1522902252123343128FF9AD7F
:10BF1000347C00D39DEE9C4009EF9DFFEE9C8FF09A
:10BF20008003E4F5F0121C3D902252123343121CA0
:10BF30001245F024FFB322C454F0FEEF4E22FF90CE
:10BF40002614121E71E9240622FF121E71E924082C
:10BF5000F9E43AFA22121E71E924DAF9E43AFA74A1
:10BF60001A75F052021C3D121E71E9240522740755
:10BF700075F0D0021C3DFF0921B3E0540F222417B5
:10BF8000F9E43AFA744022FF74017E00A8070822FF
:10BF9000F582E43412F583E022D223D2247182EFB9
:10BFA000222418F9E43AFA7D04E4FF227886E6FFB9
:10BFB000E4FEEF30E2057440FE8008EF30E104EE6D
:10BFC0004420FEEF543824F0600724F070087F030B
:10BFD00022EE4402FF227F0122EF540F24FE60165E
:10BFE00014601714601824037019EF30E704740408
:10BFF000800E7401800A7402800674038002740546
:10C00000121B1522902008E0D394004008E014F0A1
:10C01000D394005006129F3812802122E49020030E
:10C02000F022E4902003F0EF605290210DE020E038
:10C030004BA3E0C454F0440590210DF0A3E0FF545D
:10C04000F0FEEF24FE540F4EF0EEC4540F2402FE17
:10C05000C203902002E0FF12832A24BA128322FD39
:10C0600012832A24B6128322FBC003129E1A12A343
:10C0700069902594EE117D0D03129F4022F0A37468
:10C0800081F0A37419F0A37494F022902710125534
:10C09000C912832A4AC36001D35025E924BC128304
:10C0A00022C4540FFF902710E0B5071412832A24EE
:10C0B000BA128322FF90271131FD1283226F600292
:10C0C000C322E4902714F0902710E0FF902714E09B
:10C0D000FEC39F5028902711121E71128FD5EEFFBC
:10C0E0003113121AADFD12832A24BD3101121AAD8B
:10C0F0006D6002C322902714E004F080CAD322248A
:10C100000BF9E43AFAE92FF9EE3AFA22240BF9E4B2
:10C110003AFAED7E0029F9EE3AFA229026B8EDF0CF
:10C120009026B5121E91E49026BBF0E924021283FA
:10C1300022700221EE31EF1227358F529026B51270
:10C14000B68B128322FFC4540FF54CEF540FFF90AF
:10C1500026B9E0C39FC39405404F7E009026B512D8
:10C1600087FD3105121AAD9026B51288C89026BAFF
:10C17000F0E54C704590268B12272B9026BBEFF0F4
:10C18000E054FCFFF09026BAE05406C3134FA3F02E
:10C190009026B8E075F002A42481F9740F35F07B85
:10C1A000029026BB122FF280115352FC4352019091
:10C1B00026B512BF4A7408121B15E54C25E0FF7422
:10C1C00003A807088002C333D8FCF452529026B566
:10C1D000121E71E924081283221313135403FEA8BC
:10C1E00007088002C333D8FC425231EF5104229039
:10C1F00026B8E075F002A42480F9740F22121E7193
:10C20000E924042235F07B02FEAF01AD52022FF784
:10C210009026CE121E919026D1121E717D05E4FF4C
:10C220001280049026CE121E71E92401128322FF8F
:10C230009026D1121E71EF121B159026D11255BBFC
:10C24000E4121B159026CE12BF67128322FF9026A0
:10C25000D112B68B1288CF9026CE31FD128322FFE9
:10C260009026D11287FDEF021B15518B601890208C
:10C2700009E0FEEF6E600F092003E0600C9021B32F
:10C28000E054BFB50603D38001C3229021B3E0FF81
:10C29000540F22EF54F84DFF22E94A600789828A41
:10C2A00083121F3322902644121E91902648124476
:10C2B00084FF90265AEDF0902648121E71E9240161
:10C2C00012832290265BF090264B51DD902644127B
:10C2D0001E7112A615EF7F0060027F0122E0FDA310
:10C2E000E090265CCDF0A3EDF022902662E090264F
:10C2F0005AF0902663E090265BF090266451DD02B0
:10C30000A61512832A4A600BE9240212832230E523
:10C3100002D20122EF60049021B8F0902103E0FFE7
:10C3200090200A121E717191902103EFF0604D2050
:10C33000014A902101E0C330E501D3920690121C1E
:10C34000E0FD9021B9121E7112A369902102E090C4
:10C350002594F090200DE090259571B6F090210382
:10C36000E0FB12A79F70299021B87402F090200082
:10C37000E0FEA3E0F5828E387F0280119021B8E0C4
:10C38000FF902000E0FCA3E0FDF5828C83121F33B8
:10C3900022EFC394E8501CEF9193FEEF5407FDEE9B
:10C3A000A805088002C313D8FC30E004EF04FF2284
:10C3B0000F80DE7F0022F0A37419F0A374A32290F3
:10C3C000259C1255C99025A4E05437F0E0FE542076
:10C3D000902101F09025A5E0FDA3E0902000CDF094
:10C3E000A3EDF09025A0121E719021B9121E91901C
:10C3F00025A3E0FD902102F090259D121E71902052
:10C400000A121E91EE442090200DF0E49021B8F025
:10C41000C201EDD3948240037F00227F02124C457B
:10C420009025A7129F90605690259CE0FF9025A72D
:10C43000121E71E924B61288CF9025A4E0FF30E0E7
:10C440000FE4902103F09181EF6401A371B680188D
:10C4500091819025A4E09025B0F0902000E0FFA30A
:10C46000E09025B1CFF0A3EFF09025A7918A902519
:10C47000A0121E717D027F1012BA0F7F01227F0071
:10C48000229025A3E09025AFF022121E719025B3D3
:10C49000021E91131313541FF582758300021AC6EE
:10C4A0001DED9193FFED5407FEEFA806088002C32F
:10C4B00013D8FC5401FF2290121CE0FFC003C002FD
:10C4C000C001902621121E719025A0121E91902667
:10C4D00024E09025A3F0902625E09025A4F0902656
:10C4E00026E0FDA3E09025A5CDF0A3EDF0D001D08E
:10C4F00002D00361BF902016E030E112124051904B
:10C5000002B0F0E0D394F9400374F9F0D2AD22B157
:10C5100017E49002B0F0227B017A2179AF7D04E428
:10C52000FF028004902003E0600B122F1FEF6005D4
:10C53000E4902003F022C201C205E4902003F0D26F
:10C5400003902106F0C2022275FF01E5A4C330E486
:10C5500001D322301B3543FA08301905123FFB8006
:10C5600002E4FF125032E4F5FF53B1FDF5FF43B191
:10C5700002E5B130E2FBE45FFFE5B120E30D43FCEF
:10C58000047F017E00B18EB14850FCA21B2275FFD2
:10C59000017C0C7D35121F35E47B64FAF9F8121D1D
:10C5A00002788BA60608A60718E6FC08E6FDAE048E
:10C5B000EEF5A9AF05EFF5A775FF0175A41075FF9E
:10C5C0000275F60275FF0175A4152290279FEDF004
:10C5D000A3EBF0EF607DA2EB921AC2EBD21B902787
:10C5E0009FE090183A935406900414F09027A0E02E
:10C5F000703CC219D18175FF019027A1E5DEF0756D
:10C60000FF01A3E5DFF075FF01E4F5DE75FF01F53D
:10C61000DFF5FF75CE11F5FFF5CFF5FF75CE21F5EE
:10C62000FFF5CFF5FF75CE31F5FFF5CF800D9027E3
:10C63000A0E0B40106D219D177D18390279FE0FF03
:10C64000900414E0FDE4902695F0AB1B1239D04025
:10C650002580E8A21A92EBC21BC219E4F5FF53B180
:10C66000FD123F1575FF019027A1E0F5DE75FF0172
:10C67000A3E0F5DFD181222CEBD2FBD1EE751520A2
:10C6800022D177E4F510F51475152090183E93F536
:10C690001B901841E493F513907FB2E493FFF4608C
:10C6A000028F1B907FB5E493FFF460028F13E4F5D3
:10C6B00017E5179018CA93D3951B40070517E51780
:10C6C000B40EEEE517C3940E40057517FF8007E51D
:10C6D00017C454F0F517024C0924B7F9E43AFA22CA
:10C6E00024D8F9E43AFA2224BBF9E43AFA22901861
:10C6F00032121E0C902524121E28901836121E0C81
:10C70000902528121E2890183AE49390252CF0903A
:10C71000183BE49390252DF090183CE49390252E3F
:10C72000F090183DE49390252FF0D22D90182E1202
:10C730001E0C123AF9E4F510F51422D1EE7515200D
:10C7400022902715EFF0A3EDF0A3121E919027166B
:10C75000E06047901220E06012902715E02410FF5F
:10C76000F19B902717121E71EF8017902715E06438
:10C7700001902717700712E17174808005121E71F5
:10C7800074FF121B15902718E41227E4902716E077
:10C7900014F0902715E004F080B32275FF03E4F550
:10C7A0009712CEDEE59720E1FB75FF03AF9922904B
:10C7B000274B7410F090274BE0FFD3947F503AF151
:10C7C0009B90274CEFF090274BE0B410067E1D7F26
:10C7D0000F800890274DE0FEA3E0FF7B017A2779C8
:10C7E0004C12540A04F012C81790274DEEF0A3EF34
:10C7F000F090274BE004F080BC90274DE07002A33E
:10C80000E07F0070027F01901220EFF024FF229061
:10C81000266BE4F0A3EDF09026661255C690266BC9
:10C82000122752604C902668E412274990266DF03A
:10C830007D80ED60E81171EE7C0030E7027C0190B4
:10C84000266DE05D7B0060027B01EB6CFCEF25E078
:10C85000FFEE33902666F0A3EFF0AF04EF600C908C
:10C860002666E06410F0A3E06421F0EDC313FD80C0
:10C87000C1902666E0FEA30EFF227F0F7E1D110FE2
:10C88000902672121E71902675E0FD80827B017ADF
:10C890002379D5902778121E91902778124484FF2F
:10C8A00012442A902778121E7174FF021B1512A7DA
:10C8B000977417F0EF7006A37405F080069023E5D7
:10C8C0007404F012A35E11D7E4A3F0A3F09023D96F
:10C8D000E0FB7F0102A2DB9025947403F0A37405B2
:10C8E000F0227E197FF812448ABFFF0312AFAA22FA
:10C8F00090277B121E9190277B12BF67F9E43AFACA
:10C900009025E0121E917B015119021AA29027BDB9
:10C91000E0C394042290277E121E917D2AE4FF1228
:10C92000800490277E121E7111F090277E51119085
:10C93000277E1255BB7401121B1590277E129F7320
:10C94000F9E43AFA7453121B1590121DE0FF30E01F
:10C9500008121AAD4480121B15EF7F0030E1027FF0
:10C9600080EF441CFF90121DE0FE7D0030E4027D4C
:10C9700040EF4DFFEE7E0003E5027E20EF4EFF907C
:10C98000277E12B68B1288CF90277E1287FD740106
:10C99000121B159023E2E0D3942340037423F090FC
:10C9A00023E2E0FE240790240DF0AF0690277E12CC
:10C9B0003343C003C002C001902380121E71128F46
:10C9C00036D001D002D003028F42300E3A200F370A
:10C9D000510AEF70327B017A2279593115E49022A5
:10C9E000551255EFF0A304F0FB7A22795590240DEF
:10C9F000E02404902652F074111255E8F090121CB5
:10CA0000E0FF7DFF0288D77F00227E007F0402279F
:10CA10003C121E717401021B157A2379809025E364
:10CA2000121E917A2379E29025E6121E917A1279EC
:10CA30001D229024107401F0E4A3F09023B304F0BD
:10CA4000E4A3F09023DB7424F0A3740EF09023DAB7
:10CA50007401F0EF60117B017A2379E89025E012F0
:10CA60001E915119121AA212A1B7E4902379F0C2B3
:10CA70000EC20FC210C211FFEF700241FED21E7132
:10CA800023AD07ED6401707890121AE0901219F04E
:10CA9000E4A3F090121FE090121EF0901218E090A4
:10CAA0001217710B74017E00A805088005C333CEF0
:10CAB00033CED8F9FF90121BE0FCFBEF5B6006EC75
:10CAC0004401F0800790121BE054FEF090121BE02E
:10CAD000FF7401A805088002C333D8FCF45F9012EC
:10CAE0001BF0E4FD74272DF582E43412F583E0FF9A
:10CAF00074232D12AD35EFF00DEDB404E722C21E04
:10CB0000229025D2E0FF5178D22622F0901216E032
:10CB100014F0227123EFF46009201E0612AD3DE4EB
:10CB2000710B227E02EF6017901216E060117418EC
:10CB30002E12BF90B50706C3EE9401FF22DEEF7FF1
:10CB4000FF229023E1E0FF22D20D1255CF79B612D9
:10CB5000900312A0AA715C02B75DEFF07E007F0720
:10CB600012273C9023E1EFF0229027A7EEF0A3EFED
:10CB7000F012B75D9027A70EFCA3E0FDE4FF02A52D
:10CB8000759026D4121E919023E1E0600512A7282B
:10CB90006002C322E4FFEFC39D500E9026D4121E04
:10CBA00071E92F128322FE80027E00744D2FF8A6B9
:10CBB000060FEFB405E071D212AFEC7405F012313C
:10CBC0001E9026D8E0FCA3E0FD7F0112A575EF249E
:10CBD000FF227E117F527B007A00794D229012163F
:10CBE000E0B40207301E047F0180027F00227F0232
:10CBF000E4901216F074182FF582E43412F583E4F1
:10CC0000F0DFF222902723E0FEC394025027EE25A6
:10CC1000E0241FF582E43427F583EFF0AF05902779
:10CC200023E0FE04F0EE25E02420F582E43427F52D
:10CC300083EFF0D322C322AD077F0480C79027C5BE
:10CC4000EFF0902723E0602D90271FE0FF9027C58D
:10CC5000E0F8A607902720E0A805F67B017A27795F
:10CC600021128F367A27791F7F02128F4290272355
:10CC7000E014F0D32290275CE0F8E4F6C322E4FF4E
:10CC8000128FCDF8E6FC08E64C601A128FCDF8083A
:10CC9000E616187001161486044C700991F676FF9A
:10CCA000EF91ACE4F60FEFB402D622EE25E025E0DA
:10CCB0002436F82290121CE0B50702D322EF70024E
:10CCC0007FEFE4FEEE128FCEF8E6FA08E64A601F28
:10CCD000EFB4EF0891ABE6B4FE02D32291ABE6B518
:10CCE000070DEE91F7E66D6004EFB4EF02D3220E6C
:10CCF000EEB402D0C322EF25E025E02437F822EF7E
:10CD000070027FEF9027C774FFF0FDFCE4FEEE1287
:10CD10008FCEF8E6FA08E6FBD39DEA9C5006AC02FB
:10CD2000AD03A90691ABE6B50704A9068016EE127D
:10CD30008FCEF8E6FA08E64A70059027C7EEF00EA7
:10CD4000EEB402CAEEC3940240109027C7E0FE94EE
:10CD5000FF5002A906E991ACA607AF0122E4FFEF5C
:10CD6000B16BE060050FEFB402F52275F04BA4241F
:10CD7000BCF582E43421F538227B017A2779B002B0
:10CD80004441E4F530EF24FF9213EF60028002800B
:10CD9000E89027AF7478F07B017A2779B07C1A7D10
:10CDA0003490268974FAF0A37478F002444B9027EB
:10CDB000AFE014F07004C213B179221DEDB1E2129C
:10CDC0008322FFED5407B1DB8002C333D8FC4F024E
:10CDD0001B1590121BE0FF90271EE0FE7401A806B1
:10CDE0000822131313541F29221DEDB1E2128322CE
:10CDF000FFED5407B1DB8002C333D8FCF45F021BA4
:10CE000015ED600CE4121B150429F9E43AFADDF47F
:10CE100022E4FFED601A7E01EE600C121AAD5E6036
:10CE2000010FEE2EFE80F1740129F9E43AFADDE6F5
:10CE30002212832A4AC36001D34002C1BC12832A52
:10CE40001255BF74FF121AF3121AADD394014002A7
:10CE5000805C12832A24011283226401705612839B
:10CE60002A128801128FF954076403704112832A31
:10CE700024B6128322FD90211CE06D703112832AAA
:10CE800024B712832220E72612832A24B912832290
:10CE9000D394405019200F1612832A12880112BA17
:10CEA0000312832A24B71283224410121B15129FE7
:10CEB0008A024CC7E49026E4F0128021229026E5F5
:10CEC000E0600314F022129F38C13175FF0375979B
:10CED00001D1DEE59720E1FB75FF03AF992275FFD5
:10CEE000038F9875FF0322F11875FF03121AADF531
:10CEF000D375FF03900001F10F900002F10F900035
:10CF000003F10F75D40175FF03E5D55402FF22121A
:10CF10001AC6F5D375FF032275FF0375D40222F1FB
:10CF20001875FF03E5D5F45402FF2275FF03EF5493
:10CF30003F4480F5D1E5D520E20AE5D520E005E5BE
:10CF4000D530E1F1E5D55403FF75FF0375D50580B4
:10CF5000C775FF03ACD5EC20E13C75FF03ED543FF2
:10CF6000F5D175FF03E9F5D375FF03EA540FFF9080
:10CF70002728E0C4547044084FF5D2E5D520E205D7
:10CF8000E5D530E0F6E5D55401FC75FF0343D40246
:10CF900075FF0375D505AF042275FF0375D404E44E
:10CFA000FBFD7F0112396FE4FF1239BC75FF01757B
:10CFB000D30175FF0275D28075FF0243E704E4FFD9
:10CFC000FE0FBF00010EBE03F8BFE8F575FF025368
:10CFD000E7FB7F01122FD480FE75FF03AFD52290AF
:10CFE000271CE475F001021BFC12ADA0EF75F004E4
:10CFF000A4FD229027BCE0FF902015E022FD12AD99
:10D00000A0EF25E0FFAE01EEA807082225E04410BE
:10D010007886F622E0C454F07881F608E622FEAF66
:10D02000017B007A0079829026C17404F022C454F6
:10D030000FFD7C00EF240BF9E43EFAE92DF9EC3A00
:10D0400022C4540FFF7E00121E71E9227B017A2256
:10D0500079869025BC7419F0A37440F0E4A3F0A382
:10D060002275F04BA424BCF9742135F0FA7B0190B1
:10D070002283021E9124099FE43AFAE9229025D6E0
:10D08000E09026B9F022E49023B0F09023DA042255
:10D09000E0902595F0A3741AF0A3740CF0224403D9
:10D0A000121B1590201622121AADFF90121CE022BE
:10D0B0009023D404F0E4902383F0A3F0FF2224090A
:10D0C000F9E43AFAE4F5F0021C3D25E024AFF582DC
:10D0D000E43421F583E02290261B021E71121E719A
:10D0E000E9240A2224B9F9E43AFA227A2179B47FB0
:10D0F00004028F42FDC4540FFCED540F22F9E43AB0
:10D10000FAEF7C00292275F00A842406FD22FF54E0
:10D11000F0C4540FFE22FFFFFFFFFFFFFFFFFFFFE2
:10D12000FFFFFFFFFFFFFFFFFFFFFFFFFFFFFFFF0F
:10D13000FFFFFFFFFFFFFFFFFFFFFFFFFFFFFFFFFF
:10D14000FFFFFFFFFFFFFFFFFFFFFFFFFFFFFFFFEF
:10D15000FFFFFFFFFFFFFFFFFFFFFFFFFFFFFFFFDF
:020000040001F9
:1000000012AF226005755B088003755B017E607F1F
:100010000012196CEF6442600C12983F7E607F2FD3
:10002000E4FD1219711298CE9022ADE09022BD60CD
:10003000057403F080037401F090230E749AF0515C
:10004000B2435A1051371297385137435A20855AC4
:10005000B0C20B12958A506590230EE0FF129049B2
:10006000402D12AFB51290454025D20B90230E744F
:100070009AF0FF129049407112AFB5129045400FAF
:10008000E4FD7F02129665E490230EF01294F8903E
:10009000230EE060527F041290497FC012AFB2E09D
:1000A000FF1290497F011290497F4012AFB2E0FFEA
:1000B000129049E4FF1290491294F8802A1294F8A1
:1000C000E4FD12972251371297385137300B0A51FD
:1000D0002E129918535ADF800C51B2435A105137DF
:1000E00051B2535AEF5137200B4512958A7F521265
:1000F0009049500F7F801290497F091290491294C5
:10010000F8802C1294F87D017F0512972451371244
:1001100097385137300B0A512E129918535ADF80F5
:100120000C51B2435A10513751B2535AEF51371252
:10013000ADB890236EE06403701C7D037F011296BE
:100140006512B164AD07EDC394FF500A7E607F2F46
:10015000ED04FD1219711238E37F012290278AED18
:10016000F0EF2457601824A96002410E12AF1570F9
:100170000612983F02ADFB0922BD7403F0229022C3
:10018000C4E064EE706030084590230DE014F0E0A8
:1001900064027020902326745A12AECC129911EF8B
:1001A000600512991180027FFF12AEB2740212AE86
:1001B0008902199E90230DE064017052121A2012D8
:1001C000983F1238E390230D740A510F80FEE4FD2E
:1001D000FCFF121A1112AF159022BD700404F080BA
:1001E000277403F080229022C4E07C1A7D757F0280
:1001F000B4E90D121A11121A399022C474EE800754
:10020000513E9022C474E9F090230D740AF022F05C
:1002100075FF01435640435A40855AB08556CB7509
:10022000FF01435680435A80855AB08556CB75FFEF
:1002300001435620435A20855AB08556CB22121AC4
:1002400011E4FBFAFD7FFF021A02E5907F0020E136
:10025000027F019027C9EFF0E4FF0FEFB464FB9039
:1002600027C9E07044902370E0603E90236FE02443
:10027000FE60101460141406192403701EE4FB5170
:10028000FC800B7B01E451FC800CE4FB71057F03D7
:1002900080067B0171057F0512966590236FE0044F
:1002A000F0E0D394044002E4F09027C9E09023707A
:1002B000F02275FF0143561022E5B054809023715F
:1002C000F012972651371297385137300B2DE5B081
:1002D000300B055420FF80035410FF902372EFF081
:1002E000300B0A512E129918535ADF800C51B24329
:1002F0005A10513751B2535AEF513722FD7F011234
:1003000019BC7D01227D017F011219BC7D0222747E
:1003100003121B159025E0121E717407121B159015
:1003200025E01255BB7401121B157BFF7A2379144B
:10033000C003C002C0019025E3121E71121EBA90C4
:1003400025E6121E71740F021B1590257FEFF0A396
:10035000EDF0A3121E91E49022B7F0A3F0E55B64E8
:10036000017003029022902581124484121F098398
:100370009A2084923184FD338941598D0F5E87C064
:100380007083E0718916728F6F738C37778D277A3F
:1003900089CB8587948600009022E9240112AE70F3
:1003A000FF6401702A12AE67FE700C12AF3B51372A
:1003B0001297265137C165EED394634007EEF4607F
:1003C0000302902212903212AEE9855AB0E18AEF10
:1003D00064026003029022902580E09022CDF022FA
:1003E00012AE9F240112AE70FF64047051902584F8
:1003F000E0FEB40309902580E09022CEF022EEB416
:10040000041412AE9F240312AE70B4070990258025
:10041000E09022CFF02212AE9F240312AE70FE6451
:10042000076007EEF460030290229022D5EE12AE30
:100430009E240412AE7012B1289022D0F022EF64F4
:1004400006702712AE676407600302902212AE9F07
:10045000240312AE70FF600B64FE6007EFF46003CC
:100460000290227E607F0C028B9D12AE9F240112AF
:10047000AE70FFB40709905280E09022D2F022EFD4
:100480006401600302902212AE6712B1289022D359
:10049000F02212AE9F240112AE706404702712AED7
:1004A00067B4012112AE9F240312AE70FF13131321
:1004B000541FC39402500E902580E09022D6F0A3E2
:1004C000EFF0029742902580E09022D812AE9E2451
:1004D0000112AE709022DA12AE65FE9022DB12AEEF
:1004E0009E240312AE709022D9F0EF6404600302E0
:1004F0009022EE6403600302902202A86F12AE9F66
:10050000240112AE70FFB40109902580E09022F71B
:10051000F022EFB4030F902580E09022F812AE662F
:100520009022F9F02212AE9F240112AE7064056091
:1005300002C11812AE9F2402F9E43AFA1255BE1213
:10054000AF4BE49022BDF0A3E0FFF4600312442A15
:10055000E4902585F012AE67541F25E012B0DCC38D
:100560009F400302902212AFF7E92E12AE70146082
:100570000F14603B14605E41607524046002C10F7B
:1005800012AFF7EE12AF0EFAE9240112AE7090220C
:10059000FAF0A3F0A3F0600B12903212AEE9855A84
:1005A000B0805C12AF3B51371297265137801E1234
:1005B000AF04FAE9240112AE709022FAF0600E75D1
:1005C000FF015356DF8556CB535ADF8038129918F6
:1005D000435A20803812AF04FAE9240112AE709019
:1005E00022FBF0600512AEE6801B12AF3B801E12AC
:1005F000AF04FAE9240112AE709022FCF0600B12F5
:1006000094EE535A7F855AB0800512972651379041
:100610002585E02402F0A15512AE9F240112AE7090
:100620006406600302902212AE9F240312AE70FF94
:100630006402707612AE6730E63430E50B9022FA31
:10064000E0D394004016801112AE9F240412AE70C5
:100650009022FAF0D394004003E014F09022FAE0E4
:100660006003029022129918435A20028F6C12AE36
:100670006730E50B9022FA0EC394FF5016801112DA
:10068000AE9F240412AE709022FAF0C394FF500380
:10069000E004F09022FAE0700302902275FF01530B
:1006A00056DF8556CB535ADFE190EF6403706A1230
:1006B000AE6730E63130E50B9022FBE0D39400408A
:1006C00016801112AE9F240412AE709022FBF0D35C
:1006D00094004003E014F09022FBE06003029022BB
:1006E00012AF3B028F6C12AE6730E50B9022FBE03D
:1006F000C394FF5016801112AE9F240412AE709066
:1007000022FBF0C394FF5003E004F09022FBE07062
:100710000302902212AEE6807712AE9F240312AE3F
:10072000706404600302902212AE6730E62E30E55A
:100730000B9022FCE0D394004016801112AE9F244F
:100740000412AE709022FCF0D394004003E014F049
:100750009022FCE06003029022028F4612AE6730C6
:10076000E50B9022FCE0C394FF5016801112AE9F5F
:10077000240412AE709022CFF0C394FF5003E00423
:10078000F09022FCE070030290221294EE535A7F04
:10079000855AB02212AE9F240112AE70FFB4110927
:1007A000902580E09022CAF022EF6413600302904B
:1007B00022902580E09022CB12AE669022CCF022CF
:1007C00012AE9F240112AE70FFB4050F902580E099
:1007D0009022DC12AE669022DDF022EFB4081312F4
:1007E000AE97240412AE709022DDF09022DF7401E7
:1007F000F02212AE9F240112AE70640760030288DB
:10080000EE12AE9F240512AE7030E7489025857435
:1008100001F012AE9F240412AE7012B0DCD39F40E0
:100820000201CDEE24FE60121460141460161460F0
:10083000182404701A12AD45801212AD3E800D12BC
:10084000AD37800812AD30800312AD291219711234
:10085000AFFD80BE9025857401F012AE9F24041276
:10086000AE7012B0DCD39F5064EE24FE60181460AA
:10087000201460281460344204704D7E607F06129C
:10088000AE9F2406801F7E607F0712AE9F240780E4
:10089000147E607F0912AE9F240880097E607F0865
:1008A00012AE9F2409F9E43AFA801612AE9F240989
:1008B000F9E43AFA1255BE12AF4B7E607F0A12AFCE
:1008C000F7121AADFD12197112AFFD808D12AE9F95
:1008D000240512AE70FF20E60302902212AE972488
:1008E0000412AE709022DDF09022DFEFF02212AE03
:1008F0009F240112AE706404600302902212AE675E
:10090000FF12AE9F240312AE70FD12AE9F2404129C
:10091000AE70FB02AB9B12AE9F240112AE70FFB40F
:100920000408902580E09022C7F0EF64066003027F
:100930009022902580E09022C812AE669022C9F0E5
:100940002212AE9F240112AE70FFB4011C12AE67DA
:100950009022E5F064016008E064026003029022E6
:10096000902580E09022E7F022EF6403702D12AE14
:100970009F240312AE709022E512AE659022E6F03D
:10098000EF6401600D12B0FB6008A3E020E60302F3
:100990009022902580E09022E8F02212AE9F240160
:1009A00012AE706405600302902212AE9F240312FF
:1009B000AE709022E5F064016008E064026003021A
:1009C0009022902580E09022E9F02212AE679022DA
:1009D000E512AE9E240112AE70FFB4050990258089
:1009E000E09022E1F022EFB40209902580E090220D
:1009F000E0F022121AADFFB40B09902580E090229E
:100A0000E2F022EF64046002615A9022E5E0147083
:100A10000241B014700241D424026003029022907B
:100A20002584E06403700B7E607F01FD121971E480
:100A300041DC12AE9F12AF45E4902585F012AFD194
:100A4000400302902212991190258B124484B5071D
:100A500003129908E4902586F012B07A5047902549
:100A60008B124484FE74B02F12AEDEE06E703190B3
:100A7000258612AEDBE4F0FE1460101460131460DF
:100A8000162403701B7E607F0280107E607F0380CF
:100A90000A7E607F0480047E607F05E4FD12197188
:100AA00012B0F480B490258C12AD1A12AFFD808D77
:100AB000902584E0B403067E607F01802D12991199
:100AC00012AE9F240312AE706F60030290227E600C
:100AD0007F0161A5902584E0640370119022B0121B
:100AE00055EFF07E607F0212991FE461A512AE9F60
:100AF00012AF45E4902585F012AFD1400302902259
:100B0000E4A3F012B07A504790258B124484FE740F
:100B1000B02F12AEDEE06E703190258612AEDBE4AF
:100B2000F0EF1460101460131460162403701B7E21
:100B3000607F0280107E607F03800A7E607F048079
:100B4000047E607F05E4FD12197112B0F480B49048
:100B5000258C12AD1A12AFFD809E9022E5E0FF6455
:100B6000016008EF6402600302902212AE9F24012C
:100B700012AE70640160032090229022E5E024FE12
:100B8000602704600302902212B1545003029022A5
:100B9000129911EF60030290227E607F0112AE9FD6
:100BA000240312AE70FD021971902584E0D39407DE
:100BB00040037407F012B154500302902212AE9F0A
:100BC00012AF45E4902585F012AFD1400302902288
:100BD000E4A3F012B07A505490258B124484FE7432
:100BE000B02F12AEDEE0FF6E6042EF703A902586C5
:100BF000E0FF12AEDCEEF0EF14601014601314602E
:100C000016240370277E607F0280107E607F038041
:100C10000A7E607F0480047E607F0590258B1244ED
:100C200084FD121971800512B0F480A790258C12F2
:100C3000AD1A12AFFD809112AE9F240112AE70FF6B
:100C4000B40209902580E09022E3F022EFB4050978
:100C5000902580E09022E4F022121AAD64017059D0
:100C60007E607F0D12AE6712B0E3941340037413DD
:100C7000F012AE9F12AF454E902585F0902585E08D
:100C8000FFC394104003029022902584E024FDFECF
:100C9000EFC39E500DA312AFA0FE90258B1244848B
:100CA000800890258512AFA0FEE4FD1219719025F1
:100CB0008C12AD1A12AFFD80C312AE9F240112AE8A
:100CC00070640460030290227E607F1E12AE671281
:100CD000B0E3941340037413F012AE9F12AF457E3D
:100CE000607F1F124CAC90260FE4F0A3741012AF7B
:100CF0005A1219767E607F1F12AFF7902584E02488
:100D0000FDFD90260FE4F0A3ED12AF5A0219761202
:100D1000AE9F240112AE7064016003029022902500
:100D200080E09022D1F02212AE9F240112AE70FF1B
:100D3000B40109902580E09022FDF022EF64037059
:100D40006B902580E09022FE12AE66700C12AE9F72
:100D5000240312AE70641E60079022FF74FEF0221E
:100D6000E55BB402069022ADE070079022FF74FFAD
:100D7000F022902325E0FF21442AE49022C4F0755C
:100D80005B1112AE9F240612AE70FE12AE9F2407B6
:100D900012AE70FDED90230712B11A902305741D59
:100DA000F0A3740FF09022FEE0A3F02212AE9F2475
:100DB0000112AE7064066003029022902303740A4D
:100DC000F0A3740312AE66547FFD9022C5E06D70EF
:100DD00001E4600302902212AE9F240312AE70FF62
:100DE0009022C6E06F7001E460030290229025819A
:100DF000121E71902584E0FF12540AEFF07F0F7EDF
:100E00001D1219D0902587EEF0A3EFF0902587E012
:100E10007002A3E06002E14B12AE9F240412AF47C0
:100E2000902305E0FEA3E0FF12B0ED125409EDF0AF
:100E30001219D0902305EEF0A3EFF0902309121EB3
:100E400000EFC39477503B902584E02F24FAD3948D
:100E500077402FEFFD12AFF7E92477F9E43AFAC3B0
:100E6000E99DF9EA9400FA121AAD902586F0E0FEA9
:100E7000540FC454F0FDEE45F0FEC4540F4DF01273
:100E80001B1512AFF712B0EDFD7C00C004C0059039
:100E90002309121E0090262D121E28D005D0041200
:100EA000514D902585EFF0902309121E1C12B0EDD4
:100EB000FF125402902309121E289022C512AD1A67
:100EC00012AE6720E702E154124425E4902587F032
:100ED000A312820F12B034902307E0FEA3E0FF902C
:100EE0002305E06E7003A3E06F704F12B0346036DC
:100EF0007F01125108902585EFF06019902580E060
:100F0000902301F012972612823712AEE612903E1D
:100F100012B0D5800F12ADA81294EE12AB751282EA
:100F20002E12AF3B804612ADA81290321294F153AC
:100F30005A7F12903E12AF3E803212ADA81290320C
:100F400012AF3E1282371297268021902304E014BC
:100F5000F0E06009902580E0902300F02212ADA01F
:100F600012903212AF3E1282371297260282371247
:100F7000AE9F240112AE70FFB40209902580E0906C
:100F800022EAF022EFB40509902580E09022EBF0F0
:100F900022121AAD6401703112AE67FFD39409407A
:100FA000030290221244E312AE67607612AE9F24D1
:100FB0000312AE709022EEF07E1A7F707BFF7D648C
:100FC000123FF39022EDEFF02212AE9F240112AEF9
:100FD000706404704D12AE9F240312AE70FFD39460
:100FE00009503F1244E312AE679022EF12AE9E24E6
:100FF0000312AE709022F012AE9E240412AE70FE68
:1010000012AE9F240512AE70FDEDFF9022F1EEF0BE
:10101000A3EFF0E49022F5F0A3F0902580E0902279
:10102000ECF02275FF015356BF8556CB535ABF854E
:101030005AB075FF015356DF8556CB535ADF855A98
:10104000B075FF01227492F0FF300B07113B53562D
:10105000DF8008535AEF113E5356EF8556CB7E0280
:1010600000DEFDEF30E705435A808003535A7F11BD
:101070003E91F100300B0A345A20113E5356DF8066
:1010800008435A10113E5356EF8556CB00300B07DC
:10109000113B5356DF8008535AEF113E5356EF85EC
:1010A00056CBEF30E605435A808003535A7F113EFA
:1010B00091F100300B0A435A20113E5356DF80084D
:1010C000435A10113E5356EF8556CB00300B071193
:1010D0003B5356DF8008535AEF113E5356EF855667
:1010E000CBEF30E505435A808003535A7F113E9180
:1010F000F100300B0A435A20113E5356DF8008435B
:101100005A10113E5356EF8556CB00300B07113B5A
:101110005356DF8008535AEF113E5356EF8556CB96
:10112000EF30E405435A808003535A7F113E91F11A
:1011300000300B0A435A20113E5356DF8008435AB1
:1011400010113E5356EF8556CB00300B07113B5321
:1011500056DF8008535AEF113E5356EF8556CBEFBA
:1011600030E305435A808003535A7F113E91F100CA
:10117000300B0A435A2011E35356DF8008435A10BC
:10118000113E5356EF8556CB00300B07113B53569B
:10119000DF8008535AEF113E5356EF8556CBEF30A0
:1011A000E205435A808003535A7F113E91F100308B
:1011B0000B0A435A20113E5356DF8008435A101140
:1011C0003E5356EF8556CB00300B07113B5356DF8D
:1011D0008008535AEF113E5356EF8556CBEF30E15E
:1011E00005435A808003535A7F113E91F100300B22
:1011F0000A435A20113E5356DF8008435A10113ECD
:101200005356EF8556CB00300B07113B5356DF800A
:1012100008535AEF113E5356EF8556CBEF30E00599
:10122000435A808003535A7F113E91F100300B0ADC
:10123000435A20113E5356DF8008435A10113E5343
:1012400056EF8556CB00300B07113B5356DF800815
:10125000535AEF113E5356EF8556CBF12612823783
:10126000F1381282377E0400DEFD300B0A435A202B
:10127000113E5356DF8008345A10113E5356EF8505
:1012800056CB7E0400DEFDE5B030E704E4FE8002CC
:101290007E01300B07113B5356DF8008535AEF1184
:1012A0003E5356EF8556CBEE24FF22EFF0C232E4D8
:1012B000FF300B07113B5356DF8008535AEF113EA6
:1012C0005356EF8556CBF126128237F1381282370A
:1012D000300B0A435A20113E5356DF8008435A1000
:1012E000113E5356EF8556CBE5B030E704EF44800E
:1012F000FF300B07113B5356DF8008535AEF113E66
:101300005356EF8556CB7E0400DEFD300B0A435A60
:1013100020113E5356DF8008435A10113E5356EFBA
:101320008556CBE5B030E704EF4440FF300B0711A2
:101330003B5356DF8008535AEF113E5356EF855604
:10134000CB7E0400DEFD300B0A435A20113E53567B
:10135000DF8008435A10113E5356EF8556CBE5B057
:1013600030E704EF4420FF300B07113B5356DF807A
:1013700008535AEF113E5365EF8556CB7E0400DECD
:10138000FD300B0A435A20113E5356DF8008435A62
:1013900010113E5356EF8556CBE5B030E704EF44CD
:1013A00010FF300B07113B5356DF8008535AEF11E3
:1013B0003E5356EF8556CB7E0400DEFD300B0A43CC
:1013C0005A20113E5356DF8008435A10113E53569F
:1013D000EF8556CBE5B030E704EF4408FF300B074C
:1013E000113B5356DF8008535AEF113E5356EF8599
:1013F00056CB7E0400DEFD300B0A435A20113E53CB
:1014000056DF8008435A10113E5356EF8556CBE500
:10141000B030E704EF4404FF300B07113B5356DFB5
:101420008008535AEF113E5356EF8556CB7E040089
:10143000DEFD300B0A435A20113E5356DF8008432D
:101440005A10113E5356EF8556CBE5B030E704EF06
:101450004402FF300B07113B5356DF8008535AEF0D
:10146000113E5356EF8556CB7E0400DEFD300B0A4D
:10147000435A20113E5356FD8008435A10113E53E3
:1014800056EF8556CBE5B030E704EF4401FF300B53
:1014900007113B5356DF8008535AEF113E5356EF66
:1014A0008556CB303207535A7F113E91F17E0400AE
:1014B000DEFD300B0A435A20113E5356DF800843AD
:1014C0005A10113E5356EF8556CB7E0400DEFD3098
:1014D0000B07113B5356DF8008535AEF113E53560A
:1014E000EF8556CBF126128237F13802823775FF2D
:1014F0000153567F8556CB22300B07113B5356DFE5
:101500008008535AEF113E5356EF8556CB435A800D
:10151000113E91F17F02F130535A7F113E91F17FDC
:1015200002F130300B0A435A20113E5356DF800837
:10153000435A10113E5356EF8556CB7F02F130438C
:101540005A80113E91F1F126128237F1381282371A
:10155000300B0B12822E129918535ADF800F128211
:10156000B2435A101282371282B2535AEF128237A4
:10157000E5B0300B055420FF80035410FFEF7002DC
:10158000C322E5B0D320E701C322300B0A435A201F
:10159000113E5356DF8008435A10113E5356EF85D3
:1015A00056CB435A80113E91F1F126128237F13821
:1015B0001282377F01F130E5B020E702C322E5B0A7
:1015C000300B055420FF80035410FFEF7002C3223C
:1015D000535A7F113E91F1E5B030E702C3227F03F9
:1015E000F130D3229022AE122752707830070B12BE
:1015F0008210C207AF05FEFC805D9022BDE024FE94
:10160000602C14601B14604214603F24047042126A
:10161000AEE6113E91F1535A7F113E12B0D5802EA5
:10162000113212AEE9113E91F112AB758023902375
:101630000DE0C3940550061123F129800B91EE12A1
:10164000AB7512822E12AF3B80041123F129128256
:1016500037D2077E007C007D64121B499022AEEEDB
:10166000F0A3EFF0229026E6EFF0A3EDF09026E94C
:101670007403F09026E6E00926E8F09026E8E0D32F
:10168000940040739026E7E0FF6401700FF126128A
:10169000823712AEE6113E12B0D5802FEF64027091
:1016A0000D91EE12AB7512822E12AF3B801DEF64CE
:1016B00003700E113291F1535A7F113E12AF3E80EA
:1016C0000A113212AF3E128237F12612823712B15E
:1016D00021F012B08C12AD1A12B06C40F5128210CB
:1016E00012B121F012B08C12AD1A12B06C40F5900C
:1016F00026E8E014F0808412B121F012B08C12AD13
:101700001AC39026EBE094889026EAE0941340EB0D
:101710001226B69026E9E014F0E0D394004002C10E
:1017200073227F03D16575FF01435680435A80229F
:10173000EF6004001F80F92275FF01435680535A61
:101740007F22E490278DF0A3F01282B990230EE05F
:10175000440190278FF0B18A4002E1DD90278FE0AD
:10176000FF11495078D23251AF90278F51AB90275B
:101770008DE4F0A3EFF0918F90278FE0FE90278DFE
:1017800012AB7E90278DE0FEA3E07803CEA2E71394
:10179000CE13D8F890278D12B11A7C007D12121B3F
:1017A00049EF7804CEA2E713CE13D8F82440FFEE19
:1017B000340190278DF0A3EFF07E607F0A12196C40
:1017C000EF3395E090278D8FF0121BE690278DE088
:1017D000FFA3E090230FCFF0A3EFF0800291F890E9
:1017E0002371E0600CF126128237F138855AB080FF
:1017F00008535A7F113E53567F8556CB300B3F908E
:101800002372E06022300B0B12822E129918535A69
:10181000DF800F1282B2435A101282371282B25303
:101820005AEF855AB08014300B0812903B5356DFA4
:101830008009535AEF12903E5356EF8556CB227EC5
:10184000607F007D4212197131087E607F02E431B1
:101850001FE4FD12197112AD4512197112AD3E123D
:10186000197112AD3712197112AD3012197112AD12
:10187000291219717E607FB0E4FD1219717E607FBC
:101880000C7DFF1219717E607F0DE4FD1219717ECF
:10189000607F0E7D451219717E607F0F7D5A12198F
:1018A000717E607F107D4D1219717E607F11E4FDA5
:1018B0001219717E607F1EE4FD1219717E607F1F18
:1018C000E4FD1219717E607F20E4FD1219717E60C3
:1018D0007F0212196C9022B0EFF07E607F03121924
:1018E0006C9022B1EFF07E607F0412196C9022B2EE
:1018F000EFF07E607F0512196C9022B3EFF07E60EE
:101900007F0612196C8F5C227E607F01E4FD021954
:10191000717E607F0102196C75FF0143562022FD24
:101920001219717E607F03E4FD1219717E607F04DD
:10193000E4FD1219717E607F052290231FE0B4FF41
:10194000107E1A7F7F7BFF7D64123FF390231FEF91
:10195000F0E59030E11F9022B5E0FF603AEFB4016E
:101960000C300809E49022B5F0C208802A9022B514
:10197000E014F0802290225BE0FF64146019EFB461
:10198000130F20080C9022B57414F0D208D20980ED
:10199000069022B5E004F0E55B121F0999C4019995
:1019A000DB0299FC089A27099A880A9A9B0B9AB934
:1019B0000C9B1B0D9B5F0E9B71119B93129BC7137E
:1019C00000009BE49022ADE0600A755B08E4FD7FB7
:1019D0000412966520090261F261139022C4E0604E
:1019E0000261F29022ADE0600B755B089022BD743D
:1019F00003F061F2755B0112ADFB61F23009081270
:101A0000ADAF12ADCF8018E59020E01312AFABEF71
:101A10006005755B098003755B0BE49022B4F09060
:101A2000230D740AF061F29022B6E0600261F212B6
:101A3000AED8E0604490232612B0CEF07E607F07DF
:101A400012196C902328EF12AED012AED8E0FF121C
:101A5000AEB27403F0A3741012AE8D12199E12AEC2
:101A6000D8E0FF9022ADE06F700F12903212AEE915
:101A700012903E1294F112BA7512B17B64046002A6
:101A800061F2755B0AF061F29022B6E0600261F2E9
:101A9000311112B04BF0755B0B61F2755B0CE55CBC
:101AA00060089022C112B18361F2E49022C1F090EB
:101AB000231E740AF0C20C61F2E55C6020E5902000
:101AC000E0089022C1E55C12B1839022C1E0703E33
:101AD00012AFABEF70028033755B0D8022E5902072
:101AE000E00B90231EE0C394075002D20C90231EFB
:101AF000E0701B300C1512AFABEF600A755B09E4A8
:101B00009022B4F08008755B0B8003755B08200998
:101B10000261F212ADAF12ADCF61F29022B6E06079
:101B20000261F212AED8E0FF60269023267420F006
:101B3000740112AEA77403F0A3741012AE8D1219C3
:101B40009E12AED8E0FF9022ADE06F7003128210BB
:101B500012B17BC39404500261F2755B0E61F29086
:101B600022B6E0600261F2311112B04B74DEF080F7
:101B7000791238F09022C04701F09022BEE0FFF4C5
:101B8000600312442A12ADBE9022BD7404F0755B4E
:101B900012805F9022C0740FF09022BD7405F09007
:101BA00022C5E4F0A304F0E4902309124C20125063
:101BB00082BF010512AD558009755B089022FF7444
:101BC000FFF0755B13802B9022BEE0B4FF08200A63
:101BD0000512ADA8801C300A199022B6E0701312CD
:101BE00038E380FE9022ADE06005755B08800375E8
:101BF0005B019022B6E0600302A7439022C7E0FF9A
:101C00006024747212AF9412B14CE4A3F074041205
:101C100055E80412AEAB740812AE8912199EE49016
:101C200022C7F002A7439022C8E0603390232674B5
:101C300072F0740712AFDDA3742412B0BC7D047F70
:101C4000701219C612AED19022C8E0FF12AEB27463
:101C50000812AE8912199EE49022C8F002A74390A0
:101C600022CEE0FF6023747112AF94E4A3F0E55B31
:101C70007EFFB408027E00092329EE12AE77121906
:101C80009EE49022CEF002A7439022CFE06029127A
:101C9000AF51A312AFAA90232BEF12AEFA12AED01F
:101CA0009022CFE0FF12AEB2740912AE8912199ED3
:101CB000E49022CFF002A7439022D0E07002A191DD
:101CC00012AF51A3F09022D5E0FFB4FF067E077F4C
:101CD00007800090232CEFF09022D4E06407706F0F
:101CE00012AFAB90232BEFF090232D7407F07A23E3
:101CF000792F12B01E12AF64747712AD1412AF6454
:101D0000740612AD147E607F1E12AF61EF12AD1427
:101D1000E4902729F0902729E0FFC3941050247EF7
:101D200000741F2FFFEE3460FE12AF61EF121B151F
:101D300090272B124484600B12AD17902729E004E2
:101D4000F080D2902729E0240390232EF080279062
:101D500022D4E0B4DE1212B14312AFAA90232BEFCB
:101D6000F0E490232DF0800E12B143F090232BF07D
:101D700090232D74FEF012EAD112AF6C240D902640
:101D80005A12AE899022D012B0179022D0F002A73A
:101D9000439022CAE0604812B1737412F07E237F30
:101DA000111238A8902328EFF0A37404F0743612AF
:101DB000AFDDA3740AF07F02300B027F0190232D68
:101DC000EFF0E4A312AED09022CAE0FF12AEB274DC
:101DD0000B12AE8912199EE49022CAF002A743901A
:101DE00022CBE07002C16C12B1737414F09022CC5B
:101DF00012B044EF121F099E49209E2D319E3533AB
:101E00009E37599E3D5A9E395E9E39709E25719E21
:101E100039729E47739E3B779E397A9E39859E39EB
:101E20008600009E519023297403F0802990232975
:101E30007406F08021801280108004800C800A904B
:101E400023297402F0800F80009023297401F08010
:101E500005E4902329F012AED19022CBE0FF12AE20
:101E60007E12199EE49022CBF002A7439022CDE08F
:101E7000FF6034742012B0E0E5B030E50AE5B03020
:101E8000E605E5B020E70890232874FFF08005E41C
:101E9000902328F012AEAC740312AE8912199EE49E
:101EA0009022CDF002A7439022D1E0FF6027745E1C
:101EB00012AFBFA314F0A37405F0E4A312B13A1259
:101EC000B13A12AEAB740912AE8912199EE4902297
:101ED000D1F002A7439022D2E0FF601B902326742A
:101EE00071F0A37408F012B16B12AE7712199EE470
:101EF0009022D2F002A7439022D3E0FF60377471A2
:101F000012B05A9022D412B109EEB4070612B16B86
:101F1000F0800CE4902329F0A3F09022D3E0FF128C
:101F2000AEB2740512AE8912199E12AED1E490229F
:101F3000D3F002A7439022E7E06057745912B05AD9
:101F40009022E512B044EF7F06B401027F0990238E
:101F500029EF12B0BC12B0209022E5E090272BB4FC
:101F6000010B12B1107B017A22799E800912B11007
:101F70007B017A2279A712022E12AED19023291268
:101F8000B0AF12AE899022E712B0179022E7F002AC
:101F9000A7439022E8E0FF700302A01B745912B01F
:101FA000839022E6E030E6219023287482F0A37427
:101FB0000112AF5A12B0C412B007740212AEF3127B
:101FC000B0CE12AEAB741180459022E5E064017092
:101FD0001F90232804F0A312AF5A12B0C4F0A374C8
:101FE0000512AED09022E8E0FF12AEB2740A801E55
:101FF00012B0FB701F90232804F0A30412AEF374F8
:102000002012AECC9022E8E0FF12AEB2740A12AEFB
:102010008912199EE49022E8F0E1439022E9E0FF62
:102020006043745912AFC89022E512B109A374023B
:10203000F0EEB4010AA37471F0A37405F08014EEFD
:10204000B4020990232A12B0CEF08007E490232A2C
:10205000F0A3F012AEAC740612AE8912199EE49091
:1020600022E9F0E1439022E0E07002210074851241
:10207000B1319022E512B044E490232AF090272A4F
:10208000F0EF6401701B90232904F0129911EF60A6
:102090005712991190232BEFF090272A7401F080AA
:1020A0004712B0FB703D902329740412B02D902785
:1020B00029E0FFC39404503074B02F12AEDEE0FF6D
:1020C000601990272AE07C007B01242BF9EC342353
:1020D000FAEF121B1590272AE004F0902729E0045C
:1020E000F080CBE4902329F012AED190272A12B0D1
:1020F000AF12AE899022E012B0179022E0F0E143D7
:102100009022E1E0FF601A748512B063A37402129A
:10211000AEAB740312AE8912199EE49022E1F0E195
:10212000439022E2E0FF601A9023267485F0740C3D
:1021300012AEA7740312AE8912199EE49022E2F047
:10214000E1439022DCE070024148747012B0639069
:1021500022DD12B044A37401F0EF121F09A1760131
:10216000A17C02A18203A18804A18E05A194E0A212
:1021700009FF0000A2177E067F06410D7E607F07E3
:10218000410D7E607F09410D7E607F08807F7E600B
:102190007F0A807912B0BD12B0209022C112AEBC6D
:1021A00090231E12AEBC12B16412AEBEA20BE43379
:1021B00012AEBD90232212AEBC90232112AEBC9071
:1021C000232012AEBC9022BC12AEBC90272BE4752B
:1021D000F001121E7A74AA121B159022B912AEBC1D
:1021E0009022B9A312AEBC90237312AEBC9023739D
:1021F000A312AEBC9022BF12AEBC90232312AEBC81
:10220000902323A312AEBC80137E607F0B12196C47
:1022100090232AEFF08005E490232AF012AED190AB
:1022200022DDE064E090272960057405F0800374E6
:1022300014F09022DC12AF6A90265A12AE8912195D
:102240009EE49022DCF0E1439022DEE07002611017
:102250009023267470F0A3740912AF5A9022DDE027
:1022600090232AF0E4A3F07E607F0612196CEF64DD
:102270000A702F7E607F0721196CEFF4702412AD75
:102280004C643C701D7E607F0812196CBF3C137E4D
:10229000607F0A12196CBFD8099022DFE04480F0F9
:1022A00080079022DFE0547FF09022DFE090232C23
:1022B000F07A23792D12B01E7E607F0612AF61EF97
:1022C00012AD147E607F0712AF61EF12AD147E6015
:1022D0007F0912AF61EF12AD147E607F0812AF610B
:1022E000EF12AD147E607F0A12AF61EF121B151260
:1022F000AED17B017A2379269022DDE02407902657
:102300005A12AE899022DE12B0179022DEF0E1431D
:102310009022E3E06057747712B1317E607F0D1236
:10232000B0267E607F0D12196CEF6402600A12AF56
:102330009DFE12196CEF600D12AF9D12AF77F0E0A9
:10234000C3941040DD902729E0FF700712B095126A
:10235000AF8BF012AED112AF6C240390265A12AE9E
:10236000899022E312B0179022E3F0E1439022F724
:10237000E0FF601912B15C4702F0A3741CF0E4A303
:1023800012AE7712199EE49022F7F0E1439022F802
:10239000E0FF604312B15C7404F09022F912B109BD
:1023A000EEB402089022FAE0902329F09022F9E09E
:1023B000B403089022FBE0902329F09022F9E0B4C6
:1023C00004089022FCE0902329F012AE7812199EA6
:1023D000E49022F8F0E1439022E4E0605C90232650
:1023E0007477F0A37406F07E607F1E12B0267E60C4
:1023F0007F1E12196CEF6402600A12B0A2FE12195D
:102400006CEF600D12B0A212AF77F0E0C3941040F1
:10241000DD902729E0FF700712B09512AF8BF01204
:10242000AED112AF6C240390265A12AE899022E4EA
:1024300012B0179022E4F0E1439022EAE0602974A0
:102440007312B00E1244DD902328EFF09022EEE0DC
:1024500090232912AED09022EAE0FF12AE7E12192C
:102460009EE49022EAF0E1439022EBE0FD60547498
:102470007312AFC89022EF0E902328F09022F1E063
:102480007002A3E060047F02800E9022F5E07002EB
:10249000A3E07F0060027F01902329EFF09022F5F6
:1024A000E0FAA3E0FBEA90232AF0A3EB12AED0AF50
:1024B0000512AEB2740612AE8912199EE49022EB98
:1024C000F0E1439022FDE0FF6025747A12AFBF1265
:1024D000B14CA37401F0A3740AF0E4A3F012AEAA05
:1024E000740812AE8912199EE49022FDF0E1439027
:1024F00022FFE0FF603C747A12B083EFB4FF067EE7
:10250000007F01800F9022FFE07E00B4FE047F0078
:1025100080027FFF902328EF12AED09022FEE0FFD2
:1025200012AEB2740312AE8912199EE49022FFF02B
:10253000E143902300E06046747A12B0047401F025
:102540009022C512B102902329F0EDA3F09023024E
:10255000E0B4FF107E1A7F6B7BFF7D64123FF39027
:102560002302EFF012AED19022FEE0FF12AEB27461
:102570000512AE8912199E4E902300F0E14390237C
:1025800001E0FF6032902326747AF0A37407F0EF25
:102590007FFFB4FF027F01902328EF12AED090227C
:1025A000FEE0FF12AEB2740312AE8912199ED20A77
:1025B000E4902301F0E1439022D6E07002C1407420
:1025C0003112B0047401F09022D7E05418601A90D0
:1025D0002329742AF090230F12B102FF3395E09063
:1025E000232AEFF0A3EDF08031902310E024C0FF08
:1025F00090230FE034FEFE7C007D05121B497D090F
:10260000121BB0AD07AC069023297422F0ECFF3307
:1026100095E0A3EFF0AF05A3EFF012AED19022D674
:10262000E0FF12AEB2740612AE8912199E7E607F70
:102630000812196C9022C2EFF0E49022D6F0E14328
:102640009022D8E0FF7002E10A9023267431F090C6
:1026500022DAE024FD601914604F24036002E103D4
:102660009023277402F0A3740512AEAB7403C1FD6E
:102670009023277406F09022DB12B044EFB40106D9
:10268000A37403F08017EFB4030E7F03300B027FB7
:1026900001902329EFF08005E4902329F09022D8BF
:1026A000E0FF12AEB2740480549023277405F0A3A7
:1026B0007403F09022D9E05418902329701204F08A
:1026C000902322E090232AF09027297405F08016A9
:1026D000740AF090232312B10290232AF0A3EDF0A4
:1026E0009027297406F07E607F0912196C9022C32E
:1026F000EF12AED09022D812AF6A90265A12AE894D
:1027000012199EE49022D8F080399022F1E0FEA3C5
:10271000E0FF4E602EEF5407600812AED112AFE416
:10272000801A9022F3E07002A3E09022F36002800E
:102730000BE4F0A3746412AED012AFE474FFF5F0B2
:10274000121BE6F1B79022B7E0F47003A3E0F46047
:10275000139022BBE0C3940A500A90231FE0F46058
:10276000031226B69022B9E0FEA3E0FF9022B71232
:1027700055DE40031231362275FF01435508535987
:10278000F78559A08555CA75FF0143540143580187
:102790008558908554C975FF014354025358FD85EF
:1027A00058908554C912821090236EEFF0E5A07FF7
:1027B0000120E3027F00229022BDE024FE6013147A
:1027C000601814602C14602F240470327D327F64F2
:1027D000802990230DE0FDFF8021E59020E00F127D
:1027E000903212AEE912903E1294F102AB75028261
:1027F000107D117F0380047D0A7F0A1295E42290E8
:102800002303E07016A3E014F0E0600512AD5580DC
:1028100002B1A0902303740AF08006902303E01411
:10282000F0E55B64136003124425229022EEE07011
:1028300013FF1244E39022EDE0FF12442A9022EDB0
:1028400074FFF0229022EEE014F022E4FD7FA90252
:10285000815C9022C4EFF07C1A7D7512823E7E1A54
:102860007F7A7BFF7DFA123FF3902325EFF0222041
:102870000B0221761282B2355AEF1282377F011293
:1028800054509027627401F07B207D04FF1255574D
:102890007F011254617F021255347F011255197F56
:1028A0000112541E74FF9025C4F0A3F0E49025CBD0
:1028B000F0A3F09025C4E0B4FF25A3E0B4FF20C34B
:1028C0009025CCE094649025CBE0940050111254F4
:1028D000E471857F0A1297309025CBB11A80D4908D
:1028E00025CBE0FFA3E0902375CFF0A3EFF0902578
:1028F000C4E0FFA3E0902373CFF0A3EFF0E4FF1256
:10290000541E7163C374FF9FF0740F9E9025C4F032
:10291000E0C4F854F0C8A3E0C4540F48FF9025CA9F
:10292000F0902320E0FEEFD39E40089025CAE0906F
:102930002320F0902321E0FF9025CAE0FEC39F50A2
:1029400005902321EEF0902321E0FB9025CAE0C3FF
:102950009BFF7E007C007D64121B49902320E0C316
:102960009BFD121B5B7185902322F0D3946450026F
:10297000615C7464F0221228B912958A40026128C1
:102980007F52129049400241F67F88129049129579
:102990008A7F53129049D2321292AF9025C6E4F04A
:1029A000A3EFF0D2321292AF9025C6717CD23212D0
:1029B00092AF9025C4E4F0A31292AB9025C4717C31
:1029C0001294F8716C9025C5E02FFD9025C4E03E6F
:1029D0004D7008902323F0A3F041C87C007D641261
:1029E0001F35C006C007716C9025C5E02FFF9025EC
:1029F000C4E03EAB07FAE4F9F8D007D006121D0296
:102A00009025C8EEF0A3EFF0C3942DEE940050167D
:102A10007D6F718EC004715D7C007DB1121F35D059
:102A200000121C5C8028C39025C9E094409025C802
:102A3000E094005020716C7C007DC3121F35C004EF
:102A4000715D7C017DAC121F35D000121C697802CB
:102A5000121DC0802FC39025C9E094559025C8E071
:102A60009400501B7D0C718EC004715D7C007D3B19
:102A7000121F35D000121CC57802121DC08005E45B
:102A8000FFFEFDFC9025CD121E289025CD121E00C4
:102A9000E47B19FAF9F8121D029025CD121E28E4E4
:102AA0007F307E75FDFC9025CD1253FB400C9023AA
:102AB000237475F0A37430F0800E9025CD121E00A3
:102AC000902323EEF0A3EFF0902323E0FEA3E0FF9A
:102AD000D394E8EE940340089025CA7464F0800C07
:102AE0007C007D0A121B5B9025CAEFF09025CAE09E
:102AF000902322F080631294F87D027F02129724C3
:102B0000128237129738128237300B0B12822E1234
:102B10009918535ADF803F1282B2435A10128237FB
:102B20001282B2535AEF802E1294F87D021297222D
:102B3000128237129738128237300B0B12822E1204
:102B40009918535ADF800F1282B2435A10128237FB
:102B50001282B2535AEF1282371297DF22A905AAC6
:102B600006AB079025C4E0FEA3E0FF229025C6E057
:102B7000FEA3E0FF22535AF7855AB022EFFEE04E43
:102B8000F0A3E0F0229025C4EEF0A3EFF022902510
:102B9000C6E0FEA3E0FF7C00021F359027B1EDF0F8
:102BA000A3EBF0EF121F09ABC001ABDF02ABF903DF
:102BB000AC1304AC2D05AC45E0AC5AFF0000AC7A78
:102BC0009027B1E030E704B145800E9027B1E0B422
:102BD000010A7E607F06A3E0FD1219710298FE9043
:102BE00027B1E030E704B13E8177917B6002817AC2
:102BF0007E607F07A3E0FD807E9027B1E030E70490
:102C0000B1378073917B70727E607F09B121902211
:102C1000C3F0229027B1E030E704B1308059917BB6
:102C200070587E607F08B1219022C2F0229027B1B7
:102C3000E030E704B129803F917B703E7E607F0ADF
:102C4000A3E0FD80329027B2E09022C1F0E490230F
:102C50001EF07E607F2FFD1219719027B1E030E7E2
:102C6000087E607F0BE4FD800E9027B1E0B4010A7E
:102C70007E607F0BA3E0FD211971229027B1E064F3
:102C8000012290231EE07052743BF09022C1E0605C
:102C90000214F01297427E607F0812196CEF6016E2
:102CA0009022C2E0700A1299119022D6EFF08006AD
:102CB0009022C2E014F0116FB14C60249022C3E066
:102CC00070131299119022D8EFF09022DA7404F068
:102CD000A314F0800B9022C3800390231EE014F015
:102CE0009022B6E0600B14F0E070069022BBE00486
:102CF000F09022B7E0F47003A3E0F460059022B7EF
:102D0000B11A9022BCE0FF9022BBE0FED39F4003AB
:102D1000A3EEF022121B1590272CE475F001021B84
:102D2000E6A3E0FD121971E4227E607F0A7DD822BD
:102D30007E607F087D3C227E607F097D3C227E6034
:102D40007F077DFF227E607F067D0A227E607F09ED
:102D500012196CEF229022FEE0902300F0229022C4
:102D6000BFE07035A3E070289022BEE0FFF460035E
:102D700012821012442A9022BE74FFF0E55BB40167
:102D8000028078E55BB402028045E49022BDF02227
:102D90009022BF743BF0A380039022BFE014F02286
:102DA000902302E0FF12442A90230174FFF022C214
:102DB00009755B027F0111529022C07405F07E1AE2
:102DC0007F847BFF7D64123FF39022BEEFF0229060
:102DD00022BD7402F022EF70059022F5B11B902203
:102DE000F1E07002A3E0700D9022ECE09022EBF095
:102DF000E4FF1244E3E49022B6F0229022BD740175
:102E0000F022E49022B6F0EF9022BB7008F09022FE
:102E1000B7F0A3F022E004F0229026ECEFF0A3ED4F
:102E2000F0A3021E9190272EEFF0A3EDF0A3121E47
:102E30009190272FE0602790272EE02480FF121A20
:102E400057902730121E71EF121B15902731B11ABF
:102E500090272FE014F090272EE004F080D32290EA
:102E600027CAEFF022FFF0902581121E71E924029B
:102E7000F9E43AFA021AAD0F9022B6740FF07B0112
:102E80007A23792690265A7404F0A37425F0A3744B
:102E90001AF0A3748EF022902580E09022DEF0904C
:102EA0002581121E71E922A3F0E4A3F09022B674EA
:102EB0000FF07B017A23792690265A22E0FF902793
:102EC0002BE475F001121E7AEF021B15F0A37401BA
:102ED000F09022B6740FF0229022B4E024B0F58274
:102EE000E43422F5832275FF015356BF8556CB5338
:102EF0005ABF22F0E4A3F0A37431F0A37407F0E406
:102F0000A3F0A32290258B121E71902585E07E00F0
:102F100029F9EE3A22902325E0FF12442AE4902278
:102F2000C4F07B017A2279AD9026C5121E911B7ADE
:102F30000079001219629022ADE02275FF0143561C
:102F400040435A40222403F9E43AFA90258B021EAA
:102F5000919023267471F0A37405F0E4A3F0A3F01C
:102F60002212196C90272B021E71E0FF7B017A233D
:102F70007926902729E022EF12196C902729E07C0E
:102F8000007B012429F9EC3423FAEF121B1590275A
:102F900029E00422902326F0A37405F0229027292B
:102FA000E07E00240EFFEE346022F07E607F0C0293
:102FB000196C1290491294F812958A90230E22905F
:102FC0002326F0A37402F022902326F0A37406F0C7
:102FD00022902584E024FDFFA3E0C39F22A3F0A359
:102FE0007401F0229022EFE0FFA3E0FD7A1A7B89C2
:102FF0001219F39022F12290258B021E71902585E3
:10300000E004F022902326F0A37405F0A32290237D
:1030100026F0A37403F022E0FF12199EE4227B0144
:1030200090272B021E9112196C902328EFF0E49048
:103030002729F0227B017A25798712525EE43390AA
:103040002585F022E0FF902328F0229022D0EFF097
:103050009022D57407F09022D422902326F0A374F6
:1030600002F022902326F0A37406F022C39026EBF0
:10307000E094D09026EAE0490722902586E0FFC33D
:10308000940422902326F0A37404F0227FFF129769
:10309000309026EA22FE7B0174292FF9EE3423FAC0
:1030A000E422902729E07E00241FFFEE3460227B7B
:1030B000017A237926E0240590265A22F07B017AB2
:1030C00023792A22A304F0E4A3F0A37471227420CC
:1030D000F0A3740122435620435A2022FF902585F5
:1030E000E0FE22FD121971902584E0D32290258400
:1030F000E024FA22902586E004F0229022E5E064A4
:103100000222E0FCA3E0FDEC22E0FE902328F02266
:10311000121E71A801AC02AD0322FFEEF0A3EFF086
:1031200022E49026EAF0A3229022D4F0902580E0B9
:1031300022902326F0A37403F022F0A3740CF0A3D2
:10314000740722E4902729F090232E22E4A3F0A311
:10315000741EF022902584E0D394032290232674D9
:1031600033F0A3227E607F2F02196CA37401F0A3B9
:103170007480229023267468F0A3229022B4E00485
:10318000F0E022F090231E743CF02202FFFFFFFFCC
:10319000FFFFFFFFFFFFFFFFFFFFFFFFFFFFFFFF3F
:1031A000FFFFFFFFFFFFFFFFFFFFFFFFFFFFFFFF2F
:1031B000FFFFFFFFFFFFFFFFFFFFFFFFFFFFFFFF1F
:1031C000FFFFFFFFFFFFFFFFFFFFFFFFFFFFFFFF0F
:1080000003FFFFFFFFFFFFFFFFFFFFFFFFFFFFFF7C
:10801000FFFFFFFFFFFFFFFFFFFFFFFFFFFFFFFF70
:10802000FFFFFFFFFFFFFFFFFFFFFFFFFFFFFFFF60
:10803000FFFFFFFFFFFFFFFFFFFFFFFFFFFFFFFF50
:10804000FFFFFFFFFFFFFFFFFFFFFFFFFFFFFFFF40
:00000001FF
